:020000041100E9
:1030000070B500234025284C0120636101F020F9B0
:103010000223FE212800254A257401F09FF900288B
:1030200035D10223FF21224A207C01F097F90028A4
:103030002DD1204BA2899A4226D1E3891E4A934280
:103040000ED11E4B1E4963612368002B05D1002958
:1030500003D00C22200008F0EFFA01F06DF970BDEA
:10306000184A934201D00021EEE7174B174A1B681C
:10307000934205D9C02204212800920001F074FA7D
:103080000E4B13496361DFE700232374EBE7CC2287
:103090003820AC219201207401F066FA0028F3D1A7
:1030A0000C4B0D496361CFE7E462FF1FF062FF1F25
:1030B000F262FF1F5959000005830000B943001157
:1030C000A0B70011158300001863FF1F87130000CD
:1030D000ACB700119944001194B70011F7B5164B25
:1030E0000192C318021D0020009388235B05D318AA
:1030F0001B685C1C1AD09CB2402C18D88D781E0C12
:10310000AC466746CD782D023D43AE4206D10198CC
:1031100000280ED110000C70240A4C7003249BB2BE
:103120000733A343D218009B9A42DED3FEBD44323C
:10313000F9E71000FAE7C046FC0F0000802213B543
:1031400003000324019189B2520107319B18A14366
:1031500004305A1A88235B05C3181B68591C03D115
:1031600090429241104016BD99B2402907D80B00F9
:103170000733A343C0189042ECD30020F3E7443058
:10318000F9E7134B134A1B68126810B5FA249342EF
:1031900001D81A00F824104BE4021B689A4210D898
:1031A00013000E4A12689A420ED3013307D1F82356
:1031B000DB029C4203D10A49054807F0C5FF200005
:1031C00010BDFC24E402ECE7FE24E402F7E7C0466D
:1031D00000C0071100D0071100E0071100F007112F
:1031E000FFFFFF7FF0B59BB0150004900391402ACC
:1031F00000D9A0E006AB59801A80FFF7C2FF040097
:10320000042816D9002206A9FFF768FF052810D95F
:1032100006AB1B88AB420CD1002D07D0514B2A00C6
:103220000499C01807F0A0FF002802D101201BB0AC
:10323000F0BD06AB1D8020000699FFF77FFF041E3E
:103240007BD1069B0793FFF79CFF80235B01C61889
:10325000802307001B039E4201D3F826F602882331
:103260005B05F31801931B68013302D0019808F045
:103270001BF93D49019807F067FF3B1D0293331D81
:1032800005938822029B52059B181B6808935A1CC1
:103290003CD044219AB20091402A04D80320D11D89
:1032A000814389B2009103991B0C8B4224D0402AA0
:1032B00022D80122300008A9FFF710FF021E1BD1FF
:1032C000380008A9FFF70AFF0400042831D9009A42
:1032D000059B9B1880225201B218934240D288234A
:1032E0005B05C118009A09A807F026FF1D4B009A3C
:1032F00009A9F01808F0F0F8009A029B944663447C
:1033000002931A4B029AFB189A42BAD388235B05A0
:10331000FC1821680198013907F016FF200008F019
:10332000C3F8039A07AB5A8030000799FFF706FFEE
:103330000400002C03D1002079E70428FBD988235E
:103340005B05E018069907F0FFFE0323EA1C9A4389
:1033500000D16BE7034B0499E01808F0BDF865E76E
:103360000424ECE704000011FFFFFF7FF80F0000CA
:10337000F7B505001400402A21D8002701AE71805E
:103380003780FFF7FEFE042816D93A003100FFF718
:10339000A5FE042810D93688BC420BD0BD4209D006
:1033A000221CB44200D9321C064B92B2C11828002C
:1033B00007F0C2FE30B2FEBDC04300B2FBE70320FF
:1033C0004042F8E70400001137B5042204000D0064
:1033D00001A81649FFF7CCFF020004280BD1019B7E
:1033E000A34208D3AB4204D0104901A80195FFF7CE
:1033F000F9FE01203EBD0E4C23682000019308F029
:1034000053F8019920000139019107F09DFE8023B6
:103410005B01E418074B9C42EED10422034901A84A
:103420000195FFF7DFFE0020E4E7C0465555000098
:1034300000C007110000081130B589B008F02CF861
:1034400010226946254808F027F9254B009A9A4230
:103450000ED1019B029A0F2B33D80021012406982C
:10346000013B08D2002900D00292029B013331D1E6
:103470000023029325E0551CF2D102002100EFE762
:1034800010341022200004A908F006F9029B013331
:1034900001D1069B0293882304995B05C918059BFB
:1034A00006981A03120B04910592814203D02B4215
:1034B00001D108F0C1F8019B013B0193019B002B56
:1034C000DED1029B002B03D0049304984168084787
:1034D00009B030BDE025014C2D03EFE700000111DC
:1034E00050485936F7B50F490F4B0A6804001A4087
:1034F00084235B0013430B60030003271033019305
:1035000000252E00112007F03FFF084B1B683B40B1
:10351000AB4002351E43202DF4D1019B40C4A34291
:10352000EED1F7BD5CF0004000FEFEFF64F000400D
:10353000802270B5AD4CAE4BD200002120001C6043
:1035400007F0E2FF2300AB4A88331A60AA4B1A78CF
:103550006E23002A00D01133E3620A232365A74BB0
:103560001878A74BA0630138E361C3B2032B01D8DD
:1035700010232362A34B37226361C823DB00A361BE
:1035800023008C331A60082336210F3AE518E163D3
:1035900023646264E9670439251DE96725003B2639
:1035A000BC352E602500C0352B602500C4352A604F
:1035B00025000636CC352E602500083EC8352E6025
:1035C0002500D03529602100D4310B602100D8318D
:1035D0000A6021000225E0310D6025004221DC3522
:1035E000296025001B3EE4352E602500E8352B6060
:1035F0002500EC352A6022000525F43215602200F2
:10360000F0321160220018319032116022009432A1
:10361000136023003C2298331A60AF23DB00236041
:10362000794B2363032805D807F02EFE3302353784
:103630001523636096232100FA225B00A360E360F8
:10364000C8332361714BFC319200A3640A6062624B
:103650006F4A704DA2627322E2656D3A6265A2659F
:103660000232E5644A600221616696218900A16602
:10367000626709210022E166A2676749674A684ECE
:103680002167E2673560032811D807F0FDFD960831
:103690009EA61023CDE70E23CBE70C23C9E720001D
:1036A0001A259C30056020000735A03005602000F9
:1036B000A83003602300FA20F8338000186023004C
:1036C0006420A433186023005F38AC3318602300F3
:1036D0000338B03318602300C630B43318602300B9
:1036E0000020B833186023003825FC339D604D4D11
:1036F0005A665D644C4D9A64DD619625AD001D628D
:103700004A4D9A675D62F53DFF3D9D621E25484A20
:10371000DD6618675867D9651966DA67BE23C02168
:10372000444A5B00E250444B49006350043162500C
:10373000C4225200A350FA23E4205B000432A350B9
:103740000432A3503D493E4A3E4BD1603E49800081
:1037500019503E49E938FF3819503D490430195095
:103760003C491038D1613C4911633C4951633C49A3
:1037700011603C49195019003B48F83108603B4939
:10378000D16582213A4A89005A501A0039490832D3
:10379000D1671A003849B43211608821374A89004C
:1037A0005A501A00364988321160364ADA6407F0F6
:1037B000C3FE012007F080FC70BD200014259C3062
:1037C000056020000435A03070E7200010259C30F3
:1037D000056020000335A03068E720000E259C30EE
:1037E000056020000235A03060E7C0460004FF1FDE
:1037F000A465FF1F9070FF1F7845FF1F4A0AFF1F37
:103800003A07000080C3C9019A02000050C30000BB
:103810006A180000280A0000204E000088130000EB
:10382000F009FF1F0040001168100000C4090000EB
:10383000DC05000040420F0010270000FD1BFF1FA9
:10384000FC00FF1F0000FF1F252FFF1F4D32FF1F31
:10385000E530FF1FD91FFF1FF51FFF1FA121FF1F0D
:10386000491FFF1FC528FF1F8D2CFF1FD918FF1FE1
:10387000D127FF1F3925FF1F4525FF1F491EFF1FA9
:10388000011FFF1FC11DFF1FF7B50B0CFF270122F2
:10389000009300233C001E001D009446019089B255
:1038A00062469A401000084018413618B6B2FF2F01
:1038B00002D1012E00D19FB2009802401A41AD18EA
:1038C000ADB2FF2C02D1012D00D19CB20133102BDF
:1038D000E6D10320012E07D1012D04D1019B240143
:1038E000E4191C700138FEBD102EFCD10238102DD9
:1038F000F9D00230F7E710B5064C2378002B07D13A
:103900000548FFF7EFFD0548FFF7ECFD01232370A5
:1039100010BDC0466465FF1F7865FF1F6865FF1F07
:10392000F0B58BB00D0001230190102936D8FFF7B8
:10393000E2FF00231A001B48C15C01335218102B10
:10394000FAD1023B002A29D0174B184C1F680023DC
:1039500006A9E25C1600FA5C56405E540133102B57
:10396000F7D102AA07F048FD2A0002A9019807F042
:1039700063FE07F081FD23681B18236007F07CFDC0
:1039800063681B18636007F077FDA3681B18A360CA
:1039900007F072FDE3681B18E360002318000BB00A
:1039A000F0BDC0467865FF1F1844FF1F6865FF1F04
:1039B0000223F0B50124594E594D3370594B2C70E8
:1039C0001B688FB0552B10D0082006F0EFF80028A8
:1039D0000BD00023210000930420534A07F09CFDE4
:1039E0008023DB059C62FFF727FD002006F076FBB5
:1039F00007F072FBFFF79CFD07F096FB1F220124E6
:103A000000214A4B0EAF1A70494B1C70494B19707C
:103A1000494B19689143163A0A431A6060221968A3
:103A20009143403A0A431A6007F016FE07F0B4FDCE
:103A3000C120FF21414B80001A588A431A50C522E9
:103A4000920098588843BF390143995098583C498F
:103A500008408021C9010143802099509958C00530
:103A60000902090A0143995080213648490107F0AB
:103A7000FBFD03232200344901940093334807F0EF
:103A8000E3FD2C22324903A807F056FB03AC617812
:103A90002078023406F0B0F8BC42F8D101210020B1
:103AA00006F0C4F90121092006F0C0F9294B2A4A81
:103AB000196803201140A022D2020A431A60802212
:103AC000196892040A431A601968244A1140802236
:103AD00092030A431A60224B224A934200D80120E3
:103AE00007F04AFC07F068FB07F096FB307807F018
:103AF000FBFB2878C0B207F0C7FD07F0D5FA0A49EA
:103B0000042007F089FC06F0B5FA00F09FF800F0F9
:103B1000D7FD00F00BFA00200FB0F0BD4A0AFF1FDE
:103B20007845FF1F34F000403B000108480AFF1FA2
:103B3000490AFF1F680AFF1FBCF0004000E100E0D7
:103B4000FF00FFFF7C45FF1F0058FF1F7C55FF1F34
:103B5000B8B6001114F00040FF7FF8FFFFFF9FFF91
:103B60009070FF1F0080FF1F70B500252849294A6B
:103B700029484D6308CA1B051B0DED188242F9D177
:103B80000022264B8B63264B08211A628022254B8C
:103B90009205DA67244BDA688A43DA60234A12789E
:103BA000012A03D09A6822490A409A600121EE2432
:103BB0002048E40002686C438A430260DA681120FE
:103BC0008A43DA6007F058FA112007F01DFD112032
:103BD00007F02AFB184A200C0400642390420AD8FC
:103BE000FA220023D200904205D9144B0A21C018B2
:103BF00007F0A2FBC3B2124A1372124BD4801B7897
:103C0000002B04D1104B1021187807F015FC70BD63
:103C1000000005408805054000060540FF01000042
:103C200000F0004004E100E03CF000404A0AFF1FC1
:103C3000FFDFFFFF00380040B70B000030F8FFFF48
:103C4000FC62FF1F2065FF1F1463FF1F002210B5D9
:103C50001100112007F060FB10BD0000F8B5002333
:103C600001250826394F3A4C3B62E3681120AB43EB
:103C7000E360E368B343E36007F0C6FC112007F09C
:103C8000FBF9112007F068FA40232268290013434A
:103C9000236080236268DB02134380226360A36891
:103CA00007201343A360A3682A4A1340A36080231C
:103CB000A2689B0113431022A360236C93432364E7
:103CC000236C2B43236480235B003B62226B224BDB
:103CD0001A402263626B1A406263A26B1A40A263AD
:103CE000E26B1340E3631D4AE3681340E36006F0B0
:103CF0006DF82900072006F099F88021184A112054
:103D0000536C0B43536407F09FFAFD21154B164A81
:103D100089005A508023C720626B5B03134363639F
:103D2000E36880003343E360E368104A1D43104BAF
:103D3000E56019581140802212020A431A5080226D
:103D400092051A600B4B5E63F8BDC04600F0004060
:103D50003CF00040FFFFDFFFEFFFEFFFFFFF7FFFC3
:103D6000003800400000FF1F693B0011FF00FFFF0B
:103D700000E100E00000054030B503A804880B20F6
:103D8000002C0ED14968074D087849780902014393
:103D90000A20A94205D1012120001980024B1B7A7B
:103DA000137030BD192A0000FC62FF1FF7B5150023
:103DB00008AA16884A680F4F1478527812022243D4
:103DC0000A24BA4214D10122DBB2019200962A00E1
:103DD00007F0A0F8041E0BD1074B1B68002B07D07F
:103DE00068782A78000210434242504101309847D7
:103DF0002000FEBD022900008062FF1F30B50125B2
:103E000003790400BFB02B4212D00A49408806F063
:103E1000EDFB28420CD06A46074B69465B8D558006
:103E20001380064B60881B7A1371002203F0A0FCFC
:103E30003FB030BD7862FF1FC041FF1FFC62FF1F13
:103E400010B50549054806F087FB0421044A0548DA
:103E500006F044FB10BDC0467862FF1FFFFF000064
:103E6000E4B60011C041FF1F10B5024804F006FB84
:103E700010BDC046FD3D0011062383701033037151
:103E8000443B43712A3383714433C37100230222BC
:103E9000012110B503720E4B027041701C888172B3
:103EA0004472197A0273C1729A784273DA78827313
:103EB0000322C2731A7902745A7942740C228274F2
:103EC0009A79C274DB7903751123C37010BDC046A3
:103ED000FC62FF1F10B5142007F016FA124B1422D3
:103EE0000021186007F070FB002007F0ADF80120FA
:103EF00007F052F9022007F0E7F9032003F062FD12
:103F0000042005F077FD052002F0B0FF062003F045
:103F10006DFC072001F008F8082006F0BFFA092020
:103F200000F000FE10BDC0468462FF1F10B507F010
:103F30006BF9012007F090F907F0A6F8002010BDFA
:103F4000094B10B50400984205D0012904D1200086
:103F5000064906F001FB10BD0229FCD1013904F02D
:103F60004BFA0028F3D0F6E7FEFF0000AA62FF1F1D
:103F700070B50D7A100004AA2C0016881022144087
:103F8000154220D1002E20D10A78022A18D14A6881
:103F9000517815780E4A09022943914205D00D4AFD
:103FA000914209D01C800A2404E014220A491A8094
:103FB00007F042FB200070BD0C2208491A80F7E789
:103FC0001C800124F6E70824F4E70B24F2E7C0463E
:103FD000F3FF0000F4FF0000FC43FF1FC4B7001113
:103FE00010B504000749084806F0B6FA074804F07F
:103FF00085F90020E40704D50721054A054806F0A5
:104000006DFA10BDAA62FF1FFFFF0000413F0011C3
:1040100028B700110442FF1F00B5BFB06A460B4B22
:104020000B491B8801A813800A4B1A7800F07CFB0F
:104030006B4680B25880002805D0074B00226946A5
:10404000188803F095FB3FB000BDC0465E42FF1FDD
:104050008962FF1F8862FF1F5E43FF1F00B5BFB06C
:104060006A460B4B0B495B8D01A813800A4B1A78EB
:1040700001F0D4FA6B4680B25880002805D0074B77
:1040800000226946188803F073FB3FB000BDC046AC
:104090000442FF1FB362FF1FB262FF1F5E43FF1F98
:1040A000F7B50E00377A1C0008AB11003D001A88E6
:1040B00020231D401F423CD13378022B3BD1736833
:1040C0001F785B781B023B431E4FBB4208D01E4F3C
:1040D000BB4214D01D4DAB4221D00A252800FEBDA5
:1040E000002A2AD1142C2AD82200F06807F0A4FA5A
:1040F000174B1C70012CF1D9FFF7B0FFEEE7002A37
:104100001BD1202C1BD82200F06807F095FA114B28
:1041100004211C70104B187807F08EF9DEE7E3B22B
:104120000124009201940A00310006F0F3FE05001C
:10413000D4E70825D2E70125D0E70B25CEE70D25EA
:10414000CCE7C046F3FF0000F4FF000002290000A6
:10415000B262FF1F8862FF1F1463FF1F70B5160055
:1041600004AA148805AA15784A68507811780002C4
:104170002A4A0843801805284BD807F085F803130E
:104180001E29343F0720042C0BD80522121BAA42FB
:1041900000D92A0022491A803000091907F04CFA88
:1041A000002070BD0720112CFBD81222121BAA423E
:1041B00000D92A001B491A80EEE707200E2CF0D800
:1041C0000F22121BAA4200D92A0017491A80E3E7DE
:1041D0000720032CE5D80422121BAA4200D92A008A
:1041E00012491A80D8E70720032CDAD80422121BC0
:1041F000AA4200D92A000E491A80CDE70720032CD5
:10420000CFD80422121BAA4200D92A0009491A80D9
:10421000C2E700220A201A80C3E7C046DCD5FFFFB0
:1042200073B70011D062FF1F63B700115EB70011B2
:1042300059B7001154B7001110B50D21024A0348B7
:1042400006F04CF910BDC04648B700117442FF1F7C
:1042500070B500210600162005F024FE012115206E
:1042600005F020FE07F000F90400092006F074FFB5
:1042700000222B4B2B4DDA6661321A6019685B3ACB
:104280009143002E28D0023A0A431A60AC4209D169
:104290000A22DA6107321A6200221A639A63013233
:1042A000DA6370BD204A944203D11E22DA610532DE
:1042B000F1E71E4A944203D13022DA610632EAE77E
:1042C0001B4A944203D14322DA610832E3E7194AD8
:1042D0009442E1D16922F7E702220A431A6046229A
:1042E000AC4203D0104A944204D194225A6106325F
:1042F0009A61D1E70D4A944201D1E622F6E70C4AD1
:10430000944204D13422FF325A610D32F0E7094A57
:104310009442C1D1E62252005A610A32E8E7C0460F
:10432000005000400024F4000048E801006CDC026A
:104330000090D00300D8B80510B50024064B092022
:10434000DC6607F061F92100162005F03FFD210031
:10435000152005F03BFD10BD00500040F8B51C00D5
:104360000023134D0F00EB666860160007F094F809
:1043700001238022EB6623002F615200013B08D20B
:1043800006F0EAFF08200B4A1168002C03D1200038
:10439000F8BD2A61F2E72B6F034203D02B69013C81
:1043A0003370013613685B1A012BEED90124EEE756
:1043B000005000406008FF1F37B50120FFF748FF9D
:1043C0001C4D0223002101AA287CFFF7C7FF6A4683
:1043D000040002230121287C0632FFF7BFFF0443BB
:1043E000FFF7AAFF002C22D16B469A882B68D2BA1D
:1043F00053432A8910491B149B184B806B46DA885B
:104400006B6852BA5204520C53436A891B0C9B18B6
:104410000A481A1C1BB2834200DD021C130400D59B
:1044200000220B888A8001330B8020003EBD0124CE
:10443000FBE7C046E462FF1FFC62FF1F0F2700007E
:10444000002370B5124D1400EB6668600E0007F093
:1044500023F801238022EB6623005200013B08D29F
:1044600006F07AFF08200B4A1168002C03D12000C7
:1044700070BD2A61F2E72B6F034203D02B69013C28
:104480003370013613685B1A012BEED90124EEE775
:10449000005000406008FF1F37B50120FFF7D8FE2D
:1044A0001E4D07226946287CFFF7CAFF041E31D142
:1044B0006B461B787F2B2DD8FFF73EFF6B46D878D5
:1044C000F02302041B031A406B469B8814495BBA15
:1044D0009BB21A432B68000953432A891B0C9B1873
:1044E0004B806B465A789B7812031B011A436B680A
:1044F000024353436A891B0C9B181AB21B0402D552
:104500008C8020003EBD074B9A4201DC8A80F8E790
:104510008B80F6E7FFF710FF0124F2E7E462FF1F4C
:10452000FC62FF1F0F270000002370B50C4C0D002C
:10453000E366606006F0B0FF0123E366256106F0E4
:104540000BFF8020074A80001168636B034205D18E
:1045500013685B1A012BF8D9012070BD0020FCE71D
:10456000005000406008FF1F002370B5134C0E0080
:10457000E3666060150006F08FFF0123E3662661A5
:104580000F33626B1A42FCD02B0A23611023626B3B
:104590001A42FCD0EDB2256106F0DEFE8020084A0A
:1045A00080001168636B034205D113685B1A012B0D
:1045B000F8D9012070BD0020FCE7C0460050004043
:1045C0006008FF1F10B50E4C237C002B0CD0382B3D
:1045D0000BD10120FFF73CFECC22AC21207C9201C4
:1045E000FFF7C2FFFFF7A8FE10BD402BFCD1012052
:1045F000FFF72EFE0021207CFFF796FFF2E7C04672
:10460000E462FF1F10B5084B1A7C002A09D05B69D1
:10461000002B06D09847041E01D0FEF7F1FC2000C5
:1046200010BD0124F9E7C046E462FF1F10B51B4B23
:104630001A793F2A01D93F221A711979184A194863
:10464000117018221849028018480A8002804A8096
:104650009A791748802402800C208A8001324243D4
:104660002401101CA24200D9201C124AC8801080CC
:104670005A79002A01D101325A711A7A012A01D8D5
:1046800002221A725A791B7A0B4853430A21584363
:1046900006F052FE094C206010BDC0460863FF1FA3
:1046A000480AFF1F5C43FF1F2445FF1F5A43FF1F9B
:1046B000EC64FF1F5843FF1F710200001863FF1FC7
:1046C00010B507210020FEF77FFE124C002807D10D
:1046D0000C222000104906F0AFFFFFF7A7FF10BD26
:1046E0000C2220000D49FEF743FE0C2804D00C22BA
:1046F0002000094906F0A0FF094C0C2220000949BE
:10470000FEF736FE0C28E8D00C220021200006F02F
:104710005BFFE2E70863FF1FB8B70011FC0C000065
:10472000E462FF1FF50C0000F0B504000D00160058
:1047300085B0002A00D1C5E00878002120706170A2
:10474000262800D18BE00CD8072805D806F09CFD60
:104750004D28282828A09992252868D0FF23637027
:10476000A5E0712800D19AE014D8552845D05628E4
:10477000F4D17A4D0C227A49280006F05DFFFFF74C
:1047800055FF0C2277492800FEF72CFD0C2229004A
:10479000601C46E0722800D18BE0DC2800D193E059
:1047A000DB2800D0ADE0042ED8D9AA786B781202AD
:1047B0001A43EB7810271B0413432A7912061A4375
:1047C0000192052E05D0771F3A000198691D06F069
:1047D00033FF05222900200006F02EFF3A00019940
:1047E000601D06F029FF781D05E00C2220005E49BF
:1047F00006F022FF0C2005B0F0BD013A574E0C2AFE
:1048000013D8002A0AD0691C300006F015FFFFF704
:104810000DFF0C2230005349FEF7E4FC0C2231005E
:10482000601C06F009FF0D20E5E70C22EBE7013ADA
:104830004E4E0C2A11D8002A08D0691C300006F010
:10484000FBFE0C2230004A49FEF7CCFC132231005B
:10485000601C06F0F1FE1420CDE70C22EDE7434D7D
:104860001322280006F0B0FEFEF7CAFB132229002F
:10487000601CEEE712223F49601C06F0DDFE1320AB
:10488000B9E708223C49601C06F0D6FE0920B2E7D1
:1048900005223A49601C06F0CFFE0620ABE7697896
:1048A000F72900D95AE7364B188801F017FB022088
:1048B000A1E700F025FB012E02D06A78314B1A6087
:1048C00006F02AFC002096E7022A00D846E76B781B
:1048D0006370AB78A3706F781B021F43032A05D067
:1048E000033E3900B2B2E81CFEF77CFC102239000E
:1048F000E01CFEF73DFD03000330002B00DB7AE7F0
:104900002DE7DA2800D029E7042E00D826E7AB7877
:104910006A781B021343EA7812041A432B791B06A8
:104920001343082E16D9AA79697912020A43E97944
:10493000090411432A7A12060A4303921A601B687B
:10494000052229002000039306F076FE0422601D54
:1049500003A999E7FE226270F1E7C0460863FF1FD2
:10496000B8B70011FC0C0000C4B70011E462FF1FCF
:10497000F50C0000D062FF1F9844FF1FF062FF1F7C
:104980005E43FF1F34F0004070470000013870B5EF
:10499000042809D806F078FC030921081200144BFA
:1049A0000221187806F048FD70BD114B08211878D7
:1049B00006F082FD00220F4B1A71F5E700240D4B23
:1049C0000B4D082128781A681C719C7106F02CFD8B
:1049D0002100287806F080FCE6E70123054C082139
:1049E000A371034B187806F067FD00232371DBE702
:1049F0001463FF1F1863FF1F10B5002903D109209E
:104A0000013105F013FA10BD10B5084B084C988120
:104A1000D88118825882207802F0C6F80422054B0B
:104A2000012120781A7006F007FD10BD2244FF1FF7
:104A30004E65FF1F4D65FF1F10B501290DD10021E7
:104A4000092005F0F3F9054B1B78002B05D0262231
:104A5000034B04489A71FFF7D7FF10BD2065FF1F75
:104A60001863FF1FC40900000300F0B50A4D8E183B
:104A7000B14202D152008018F0BD0C782F68240991
:104A80003C5D0F271C700C7801313C402F683C5D69
:104A90005C700233ECE7C0465443FF1F10B50A4A6E
:104AA0000A49082005F0C4FA0121092005F0BEF9E1
:104AB000092005F0A7FA0121002005F0B7F9002030
:104AC00005F0A0FA10BDC046F9490011394A00119D
:104AD00010B5114B1A781870002A0ED000280BD18F
:104AE0000E4B1A78062A07D85423D340DB0703D588
:104AF0000B4B187802F058F810BD0028FCD0074B7B
:104B00001B78012B02D0033B022BF5D8044B01216B
:104B1000187806F091FCEFE72065FF1F4D65FF1F39
:104B20004E65FF1FF7B5574D2D242870FFF7B6FFD0
:104B3000FEF766FA06F028FD032253495348FFF7B3
:104B400093FF030004221C7051490130FFF78CFFD2
:104B5000302302220470437083704E4C4E4B200071
:104B6000DA8706F069FA022815D0062220004B49A0
:104B7000FEF7FEFB06280ED00321200006F084FC81
:104B80008D23E3706E3B23710622193320004349C5
:104B90006371FEF727FB0E23414F424C424E3B70A0
:104BA000013B0522300041492370043B63700196AC
:104BB00006F042FD2D2301223D493E48E371FFF7F7
:104BC00053FF01223C49FFF74FFF01223149FFF714
:104BD0004BFF0020FFF77CFF384E394A0121394B4B
:104BE0001278307801F0A2FF230000213A78307863
:104BF00001F09CFF01222178334B01391A7000200B
:104C0000019AC9B205F088FB304B1A68552A30D199
:104C100000221A602E4B3C322E489A71FFF7F4FEA8
:104C20002021287806F0C8FB0120404205F0C0FB97
:104C30000120404205F05CFCFFF7FEFAFFF700F9A7
:104C400000F084FC01204042FFF7CAF9012006F081
:104C50006BFCF72001F026F90121287806F0ECFB27
:104C6000287802F0FDF81C4806F07EFBFEF7F6FF00
:104C7000F7BDFA22084B52019A81DA811A825A82D0
:104C8000CEE7C0461463FF1F9844FF1FD062FF1F8A
:104C9000F062FF1F6509FF1F2244FF1FADAC00003B
:104CA0001C65FF1FFD64FF1FFF64FF1F73B700112A
:104CB0006709FF1F0565FF1F6609FF1F4E65FF1F80
:104CC0008643FF1F6743FF1FEE64FF1F34F0004061
:104CD0001863FF1FC40900002063FF1FF8B50A0016
:104CE00020230D001A40194239D0454B1B78002B68
:104CF00019D0444E444C327A2179531EDBB299428A
:104D000014D1FFF75FFCA379002B09D0013BDBB284
:104D1000A371002B04D1707964335843FFF774FEFC
:104D200023790133237120206840F8BD9142EAD3F2
:104D300000272771FFF766FC63790133DBB26371EB
:104D4000727A9A4202D86771FEF788FF2F4F3800B7
:104D5000FFF792F83900152006F09EFAD3E70BB260
:104D6000002B0ADA2A4B187806F0BEFB002801D087
:104D700006F0BAF980200002D6E702240E00264091
:104D8000214206D0204B01201A71FFF7A1FE20001E
:104D9000CAE70B0713D5FFF735FCFFF713FC00F04C
:104DA000EFFB194A174953790133DBB25371497A42
:104DB000994202D85671FEF751FF0820B4E710243B
:104DC0000E002640214206D00D4B1B78002BDED171
:104DD000FFF74AF8DBE70124214209D00D4800F033
:104DE00067F806F061FC3100092005F01FF8CEE7F6
:104DF000042408002040214297D0FFF70DF9C6E7B0
:104E00002065FF1F0863FF1F1863FF1F6743FF1F15
:104E10001463FF1F4C43FF1FF0B51B4B1B4F1B8838
:104E20003A8804001A4E1B4D85B09A420DD832883C
:104E30009A420AD3184B1A882B889A4205D1174AEE
:104E4000174B12881B889A421BD0052001F080F86E
:104E50003B8802AA13803388019053802B88114D20
:104E600093800F4B02A91B88D3800F4B2A78188898
:104E700002F08CFD0D4B08212878019A1C7006F079
:104E8000E3FA05B0F0BDC046EA64FF1F5C43FF1FB4
:104E90005A43FF1FEC64FF1FE864FF1FE664FF1F17
:104EA0005843FF1F4E65FF1F5E43FF1FE464FF1F53
:104EB00013B50C4B1C78002C11D1002801D00A4BE3
:104EC00018600A4A0A4B11780A4A10780A4A019275
:104ED0000A4A0092002205F017F9200016BD11249D
:104EE000FBE7C0464D65FF1FE064FF1F4C65FF1FD9
:104EF0003C65FF1F4E65FF1F2865FF1F2C65FF1FC8
:104F000010B5064B12201B78052B06D1044B13223B
:104F10001988044B187801F0F7F910BD4D65FF1F93
:104F20005E43FF1F4E65FF1F10B500240122114B89
:104F300052421870104B1C70104B1A8001F090FFF9
:104F400004220F4B21001A700E480C3206F03CFB75
:104F5000102221000C4806F037FB07220B4B1C6087
:104F60000B4B1C700B4B1C700B4B1A700B4B1C70BB
:104F700010BDC0464E65FF1F4D65FF1F5E43FF1FFE
:104F80004C65FF1F3C65FF1F2C65FF1F2865FF1F39
:104F9000FC64FF1FFB64FF1F6043FF1FFA64FF1FD9
:104FA000F8B5174C0600257806A814240078052DBE
:104FB00023D1B41F134FA5B21824BD421DD88D1F95
:104FC000ADB2BD4219D8FA256D00AA4215D21D0016
:104FD0000D4F0A3DADB2BD420FD80C4C26800C4C93
:104FE00021800C4900240A800B4A1380FFF714FF2C
:104FF0000A4B0421187806F05FFA2000F8BDC0467D
:105000004D65FF1F790C0000750C00005C43FF1F0D
:105010005A43FF1FEC64FF1F5843FF1F4E65FF1FDD
:10502000F0B50BB20D0089B0002B00DB76E1A64E87
:10503000307806F059FA041E55D00378A22B00D11F
:1050400027E1D02B1AD0912B4AD143780E2B47D190
:105050009E4B82889A4243D19D4A83681278052AE2
:105060003ED1032018567F283AD09A4B1B68002B5C
:1050700036D05B68002B33D0984731E08078072822
:105080002ED806F001F9042D1D444479ADDD637876
:10509000002B11D10622E11C8F4806F0CDFA012128
:1050A0008B4B19708D4B1A78002A5BD08C4B307863
:1050B00001F03CFD002855D00722854B1A7051E0C5
:1050C00061780029F8D1E378002B11D0854A864B0E
:1050D0001278307801F02AFD60706378002BEBD1F4
:1050E000200006F001F880200002684009B0F0BD01
:1050F000774B1B78022BF3D00121307806F04CF966
:105100000028EAD10121307806F096F9E5E76378C6
:10511000002BD1D16E4F032807D13B78052B02D14C
:1051200001333B701EE00223FBE7704B1A88704B83
:105130000293002A0BD01B78002B03D0012130787A
:1051400006F082F93B78062B04D1013BE9E7029B8C
:105150001A70F7E7042B41D10121029B30781970B6
:1051600006F06AF95B4B1B68002BB9D01B68002B5B
:10517000B6D0574A10787FE76378554F002B27D178
:105180000622211D5B4806F057FA62895A4B5B499B
:105190001A80A2895A4B1A80E3890B800521397045
:1051A00058490A80584A1380228A584B1A80584B13
:1051B0001B78012B09D11F2000F0CAFEFA229200B1
:1051C00042430421307806F03FF90022484B75E74E
:1051D000312B00D070E70022454B1A700323A0E763
:1051E00006220021434806F0EFF90023454A042136
:1051F0001380454A30781380444A138006F05CF9E6
:105200000821307806F058F9A379083B5A425341F7
:105210002F4A03331370314B1B78002B06D0344BCD
:1052200030781A78002A06D001F0BEFC0122324BF9
:1052300052421A8096E70121197006F0FDF8F5E751
:105240000821307806F038F96378002B00D047E762
:105250002C4B2E4F0293E388029A042113802A4B91
:10526000307803932389039A138063893B8006F087
:1052700093F8002800D033E7264B1B68002B00D1A1
:105280002EE7039902983A88098800881B68984796
:1052900026E74379132B00D022E70389012B0AD19B
:1052A0001D4B1B78022B06D10821307806F004F93B
:1052B000FFF726FE14E7052000F04AFE0821020051
:1052C000307806F0C1F80BE74E65FF1F05140000AB
:1052D0004D65FF1FE064FF1F2165FF1F8643FF1F11
:1052E0006743FF1F1C65FF1FFD64FF1F1E65FF1F37
:1052F0002065FF1FEF64FF1F5E43FF1FF664FF1F63
:10530000F864FF1FEA64FF1FE864FF1FE664FF1FE5
:10531000EE64FF1FDC64FF1FE464FF1F8020C001F8
:10532000014200D0E1E6CB0731D5324B1B78002B90
:105330001DD0314E05AC3378052B1AD1023B2370BA
:105340002E4B21001B7823722D4B1B7863722D4B43
:10535000187801F08FFB002809D007202A4B307005
:105360001B68002B03D01B68002B00D0984701203E
:10537000BBE60E20254B06221B7825492370254BC2
:105380001B78637002ABC01806F056F9D8E7022309
:1053900008001840194209D0174B1B78052B03D180
:1053A0001D4B188805F0E8FE02209EE604242142E9
:1053B00003D0FFF731FD200097E6082308001840CE
:1053C000194200D192E6154B1C78012C03D0022C17
:1053D0000DD0082089E6124B124A134913481B8846
:1053E0001288098800880094FFF7DAFDF1E7FFF7DB
:1053F00087FDEEE72065FF1F4D65FF1F6043FF1F20
:10540000FA64FF1F4E65FF1FE064FF1FFC64FF1F6F
:105410006143FF1FFB64FF1F5E43FF1FE464FF1F28
:105420005843FF1FEC64FF1F5A43FF1F5C43FF1FDD
:1054300010B502A804880B20002C10D14968087808
:105440004978090201430C48814209D1022119809F
:105450000A4B59881170DB7800205BB2537010BD85
:10546000074C0A20A142FAD102211980034B9988E6
:1054700011705B79F0E7C0466E2A0000FC62FF1FE6
:105480006F2A0000F7B5150008AA16884A680F4F62
:1054900014785278120222430A24BA4214D101220B
:1054A000DBB2019200962A0005F034FD041E0BD1F8
:1054B000074B1B68002B07D068782A78000210433E
:1054C00042425041013098472000FEBD02290000B1
:1054D0006065FF1F30B5012503790400BFB02B4282
:1054E00027D01549408805F081F828420DD06A463A
:1054F000124B69465B8D138002235380104B5B88EF
:1055000093806088002202F033F90E49608805F02C
:105510006DF8C0070DD56A460B4B69461B88138092
:1055200002235380064B9B8893806088002202F000
:105530001FF93FB030BDC0465865FF1F8843FF1FAD
:10554000FC62FF1F5065FF1FE243FF1F10B5074CB1
:105550000749200005F000F82000064904F0FCFF90
:105560000721054A054804F0B9FF10BDFFFF000000
:105570005865FF1F5065FF1F44B800118843FF1F87
:1055800010B5024802F07AFF10BDC046D554001194
:105590000200F0B501270A480A4E51188B1A002B59
:1055A00000DCF0BD0824157843086840384040000E
:1055B000805B013C58406D08002CF5D10132EDE7CD
:1055C000FFFF00005EB80011F0B500250F269D42D8
:1055D00000DBF0BD4C5D070944403440A400A058F6
:1055E00001357840F3E70000F0B589B06A460D0058
:1055F0000B000F27110010351C78013326002409F9
:105600003E40167054700232AB42F5D12023024A5C
:10561000FFF7DAFF09B0F0BD64B80011F0B54E78BD
:105620000B7889B036020C00170001901E43012A46
:1056300061D9974B9E4200D877E001339E421CD13E
:10564000062A17D1CA788B7812021A430B791B04E9
:1056500013434A7912061A438E4B5A6100221A707C
:105660005A808D4A5A608D4A9A608D4ADA600020CD
:1056700009B0F0BD88225205EEE78A4B9E423CD12C
:1056800084498B78002B00D0F9E00C2A31D10F220D
:10569000A3789343E278120213432279120413434E
:1056A0006279120613434B60E279A0791202024339
:1056B000207A00041043627A12060243CA60E27A3A
:1056C000A07A1202024378484A81834208D8042310
:1056D0007049142201980B7005F0AEFF1420C7E743
:1056E0001201D21889235B059A42F0D801238B70EE
:1056F000BDE7022AFAD00523EAE76C4A0123964265
:10570000E6D1FFF7FDFB052F0CD9E378A2781B0249
:105710001343227912041A4363791B061343644A24
:105720000393136005F0F8FCA1E75A4D2B78002B8A
:105730009DD1AB78002B00D1A3E02B8901339BB224
:105740000093B34200D094E0132AD4D9CF7C8B7C51
:105750003F02122120001F43FFF71AFF874200D0AB
:1057600091E0002E3ED1E378A2781B021343227908
:10577000E96812041A4363791B06134303930A2250
:105780008B4213D1FF23A370E370237163716B8984
:10579000002B0AD1E37B227C1B0212041343A27B61
:1057A000134303931B0901336B8100226B89002B88
:1057B0008DD0002A69D1686837013818000B6B69F1
:1057C00000030390984205D9686105F06DFEEB78FF
:1057D0000133EB7068681022A11C381805F07CFEBC
:1057E0002E8144E76F89009A7B1E9BB293423CD185
:1057F000E378A2781B02134322792E4E12041A4337
:1058000063796C681B0613433100042204A80393D8
:1058100005F012FF211D0C2205A805F00DFF012047
:1058200004A940421034FFF7DFFE013F012F17D1DA
:10583000039A0B232861824200D049E704223100F9
:10584000686805F049FE042203A9686805F0DCFDDC
:10585000E968039AFF23914200D139E7F73B37E724
:105860002100FFF7C1FE1034DFE70923B742A2D8B9
:105870002EE7009BB34200D9F9E6072328E702236D
:1058800026E7032324E7062322E70A2320E7C0466E
:10589000FFFE0000FC43FF1F00000111FFFF00009E
:1058A0005048593601FF0000FFFF001102FF0000C1
:1058B00034F000400844FF1F10B5034C0B000122D8
:1058C000210000F06BFA10BD795A00110B8870B5F9
:1058D00006000D000224162B11D92B0003220949C2
:1058E00000F05CFA041E0AD1074B2A881B88191C99
:1058F000934200D9111C300089B200F0EFFA200069
:1059000070BDC046A55A0011BE65FF1F10B54A788C
:105910000400013A0B000220012A07D80A78002A65
:1059200004D005222000024900F038FA10BDC0461C
:10593000D35A00110A7810B50B0004000220002A87
:1059400004D007222000024900F028FA10BDC0460A
:105950007F5B00110A7810B50B0004000220002ABA
:1059600004D009222000024900F018FA10BDC046F8
:10597000E55B001110B5034C0B000B22210000F079
:105980000DFA10BD155C001110B5034C0B000D2273
:10599000210000F003FA10BD875C001110B5034C24
:1059A0000B000F22210000F0F9F910BDE15C00119D
:1059B0000A7810B50B0004000220002A04D011223E
:1059C0002000024900F0EAF910BDC046F15C001168
:1059D000002310B51322190000F0E0F910BD0000FB
:1059E00010B5034C0B001722210000F0D7F910BDB1
:1059F000435D0011002310B51922190000F0CEF903
:105A000010BD000010B5034C0B001B22210000F05C
:105A1000C5F910BD7D5D0011F7B584890D00060044
:105A20000121002C22D000238268D3561778002B46
:105A30001EDA0C2C1AD90C3CA4B21319408800931E
:105A4000230002F076FE431E984101307B06DB0FF7
:105A50006B703F23013C1F40A4B22870AF70AC8034
:105A6000002C07D0B3680133AB6000210800FEBDF5
:105A70000020EBE7AC60F8E70B7803704B884370CD
:105A80004B881B0A83700B79C37004207047042075
:105A9000022B06D10020537811781B02009A0B4389
:105AA000138070470B8803700B881B0A4370022019
:105AB00070470420009983420AD1537810781B0262
:105AC00003430B80D37890781B02034300204B8064
:105AD0007047F8B50D004B7801240021461C037077
:105AE0002B788B4201D82000F8BD6B78B01C4F1C7E
:105AF000012B10D1890069184B88022233704B8822
:105B0000B9001B0A7370691805F096FD0436043459
:105B1000A4B2F9B2E4E7122359436B185A8804314E
:105B200032705B8810221B0A7370691805F084FDBF
:105B300012361234ECE770B5049D14001E00052BDC
:105B400001D8042070BD637812781B0213432B80A8
:105B5000E378A2781B02134302226B802A71211D75
:105B6000681D063E05F068FDB2B22A81F02AE8D829
:105B70002800A11D0A3005F05FFD0020E2E70023A8
:105B800010B50A789A4201D8900010BD9A008A1880
:105B90005488013304705488DBB2240A447094881A
:105BA00084709288120AC2700430EAE710B51100BE
:105BB000029C062B04D004201022142B01D010BD0F
:105BC000022222714B7808781B0203432380CB7892
:105BD00088781B02034363800431601D05F02CFDAF
:105BE0000020ECE710B50C788B7804315C43E4B20C
:105BF00003702200013005F01FFD601C10BD042061
:105C0000022B06D10020537811781B02009A0B4317
:105C10001380704710B50C000A88023105F00CFDA6
:105C2000208810BD70B504000D0004981100012BF0
:105C300001D8042070BD16785278120232430280D7
:105C40000200F83255701470E825002C00D10C3594
:105C5000023B9AB24280AA42EBD80231043005F0EE
:105C6000EBFC0020E6E70420009983420AD1537838
:105C700010781B0203430B80D37890781B020343F8
:105C800000204B80704710B50C000A88023105F0E7
:105C9000D3FC208810BD000070B501211E00042037
:105CA000049C0E400B4218D1CB40DDB28D4214D97A
:105CB0000A49DBB2098899420FD32300F6331D70DD
:105CC0003300580011184978165C0902314301333A
:105CD0002152D9B28D42F4D8002070BD1C44FF1F60
:105CE00010B50C000A88023105F0A6FC208810BD12
:105CF00010B50C788B7804315C43E4B20370220059
:105D0000013005F099FC601C10BD10B5110002981F
:105D1000032B01D8042010BD14785278043B1202E2
:105D200022430280CA788C781202224342809AB2BF
:105D30008280F22AEED80431063005F07DFC002086
:105D4000E9E710B50C000B8803700B881B0A437041
:105D50004B8883704B881B0AC3708A8804300631D5
:105D600005F06AFCA088043080B210BD0420012B2D
:105D700003D100201378009A1370704710B50C00FF
:105D80000B8803700B881B0A43704A880230043169
:105D900005F052FC6088023080B210BDF0B589B0C9
:105DA00003931E4B029242000700D05A019102F069
:105DB00010F81325061E2DD0029B01240370019BB1
:105DC000002B04D0001903999847001984B26B4640
:105DD0001B7A5BB2002B0FDA1021380002F00CFBAB
:105DE0001925002813D130003219E1B202F056FC17
:105DF000051E0CD10C34A4B2042304AA380005A952
:105E000093800696948101F09FFD051E02D030001C
:105E100005F0EAFB280009B0F0BDC046BC65FF1FD5
:105E200070B505000C0000280CD00020814209D07C
:105E300010222000044905F0FFFB01202B7823737A
:105E40006B78637370BDC046A4B80011F0B506004E
:105E50000D0017001C0085B002291BD0002010295E
:105E600007D1022B07D0102B03D115E00020102CF6
:105E700008D005B0F0BD69463800FFF7D1FF2A0011
:105E800069460BE069463000FFF7CAFF2200694609
:105E9000380004E0022BE9D12A003900300005F077
:105EA000A3FAE6E7031CF72800D9F72303200849E3
:105EB0009AB2013A0B80D317034006499B189B10F6
:105EC0000B80D30F04499B185B100B807047C046B2
:105ED0002044FF1F1E44FF1F1C44FF1F034B1B8851
:105EE0008B4202D3024B4000C15270472044FF1F37
:105EF000BC65FF1F014B4000185A7047BC65FF1F6F
:105F00001722014B1A807047BC65FF1F70B5050052
:105F10000E2005F069F9041E13D0D023037000236E
:105F20000622837007494570033005F085FB064B58
:105F30002100DA8A62811B7E2373044B187805F0F6
:105F4000E3F870BDD865FF1FC865FF1F7044FF1FD1
:105F5000262803D8024B4000C05A70470148FCE78E
:105F60002244FF1FFFFF000070B506000C00094D22
:105F70001C220021280005F027FB074B1E70074B51
:105F80001C7005F051FB0123002801D000231220D2
:105F90002B7070BDC865FF1F7044FF1FE965FF1FB0
:105FA00070B505000D4C0800E260A16010220021D0
:105FB000656005F009FA012803D11021A06802F0FC
:105FC00048FD10220021280005F0FEF9012803D128
:105FD0001021606802F03DFD70BDC046C865FF1F1E
:105FE00070B5041E05D1002903D006220D4805F026
:105FF00023FB0D4B1D78012D11D1002C05D1022260
:106000001A7005F0C1F8280070BD00221A70074B05
:106010001B78FF2BF7D02000FFF778FFF3E7002570
:10602000F1E7C046D865FF1FC865FF1F7044FF1F1A
:10603000030010B5002801D1002010BD00780B4AE4
:10604000002803D15988D1821B7913761378022B4B
:10605000F2D10023984200D103331370044B1B7814
:10606000FF2B01D0FFF752FF0120E6E7C865FF1FB5
:106070007044FF1F002911D000280CD04B79012853
:1060800003D140225242134303E03F22134003282E
:1060900002D001204B7170474022F4E70800FAE774
:1060A00070B5094D0100287800280BD0074C062256
:1060B000200005F0C1FA21002878FFF7DBFF20005F
:1060C00005F09AF870BDC046E865FF1FC265FF1F66
:1060D00000290AD0012808D13F224B799343C02BD5
:1060E00003D0403B5A425341981C704770B5174D3E
:1060F00006002B78FF2B15D00A2005F075F8041E3A
:1061000010D0D0230370C83B8370114B11491B780A
:106110004670C3700622043005F08EFA21002878FC
:1061200004F0F2FF0C4B1B78012B0DD10B4B1B68BD
:10613000002B03D09B68002B00D09847084B04210C
:106140001878084A05F070F970BDC0467044FF1F0A
:10615000E865FF1FC265FF1FE465FF1F1066FF1F94
:106160001466FF1F60EA0000014B98687047C04644
:10617000C865FF1F014BDB6818687047C865FF1FC3
:10618000074B10B5DA68136801331360054B1878B4
:10619000FF2803D08021C90105F04EF910BDC0468B
:1061A000C865FF1F7044FF1FF7B50E0002F0B8F876
:1061B000051E1CD00E4B06621F78002F00D10778F9
:1061C000AB791020019305F00FF8041E0FD0D023F7
:1061D0000380C73B8370019BE91DC3700622043016
:1061E00005F02AFA21003800E66004F08DFFF7BDC3
:1061F0006E44FF1F014B18787047C046E865FF1FCB
:10620000054B002805D1054B1A78054B002A00D113
:10621000014B18007047C046D865FF1FE865FF1F97
:10622000C265FF1F014B58687047C046C865FF1F15
:10623000024B1868431E9841C0B27047EC65FF1FBF
:10624000421E03000120152A03D9FF3B5A42534145
:10625000D8B27047F0B51C0000230E0085B0039043
:1062600002920B70029A934201D3002019E0E55C80
:106270005A1CD2B2002DF8D0029851198142F4DC98
:106280000233DFB2A35C18000193FFF7D9FF0028A7
:1062900007D0013D019A0399EBB233708A4202D1D3
:1062A000E01905B0F0BDDB19DBB2DBE710B50C007F
:1062B00002F08EF803001220002B03D02100588832
:1062C00004F0D2FE10BD000070B50E4D840063597D
:1062D000002B15D0186A002801D005F04DF92B5974
:1062E000586A002801D005F047F92B59986A002810
:1062F00001D005F041F9285905F03EF900232B5152
:1063000070BDC046F865FF1F1C4B70B504000E0041
:10631000150099420AD11A4B1B68002B01D112209B
:1063200070BD1B68002BFAD09847F9E7154B9942CE
:1063300015D1134B1B68002B0AD01B68002B07D00C
:106340009847002804D1104B1C70104B1D70E7E7D4
:1063500029002000FFF7AAFF0028E1D1F3E7080099
:1063600001F0DEFF0028DAD003780320A342D7D162
:106370002900300004F078FED2E7C046FEFF00009E
:10638000F465FF1FFFFF0000F165FF1FF065FF1FB1
:10639000F7B50400808801F0C3FF0025A84203D0B0
:1063A0000578A08801F0F8FF1C4E3378002B1FD031
:1063B000AB421DD11A4B28001978FFF777FF002850
:1063C00018D000233370A3790820A778A6880193FA
:1063D00004F00AFF011E0DD0D0230370CA3B837066
:1063E000019B477086808371280004F08DFE01E0D8
:1063F000002DE8D1A0880B4B8200D358002B01D090
:10640000FFF762FF1721A088FFF768FDA08801F061
:1064100017FDA08801F0EEFDF7BDC046F165FF1F36
:10642000F065FF1FF865FF1FF0B587B01D000CABCE
:106430001B88070001930DAB1B88142002930EAB41
:106440001B88160003930FAB1B880091049310ABBD
:106450001B88059304F0C8FE041E1AD0D0230370D5
:10646000CB3B47708370C670062229000430002D94
:1064700011D005F0E1F8019B21006381029B009897
:10648000A381039BE381049B2382059BA37404F0F7
:106490003BFE07B0F0BD05F097F8ECE7F7B50093C9
:1064A00008AB1B8807000C200D001600019304F0B8
:1064B0009BFE041E13D0280001F032FF00280FD0ED
:1064C0000078D0232370C93BA370009B2100238157
:1064D000019B6770A580E680638104F015FEF7BD1F
:1064E000014B1878EDE7C0467044FF1F13B5040058
:1064F00064890389C2888188C0780094FFF7CEFF41
:1065000013BD000010B5044C2068002803D005F02E
:1065100033F80023236010BDFC65FF1FA122F0B5F6
:10652000818892004A43384B384F1B6804009B18FF
:106530009D2292009B18827989B01A603B68002BDB
:106540005FD01D78324B1B68002B04D05B68002B9A
:1065500001D000209847260008363100E079FFF787
:10656000B7FD237DE0710200E0780493638A29007F
:106570000393238A0293E3890193A3880093330052
:10658000FFF752FFE378002B0BD1E289A379A188B2
:1065900002920196E27928000092012201F0CAFEDF
:1065A000E0703B68002B20D0FFF7ACFF194D287836
:1065B00000281AD0184B1978FFF778FE002814D05D
:1065C0002B78E67808200793A78804F00DFE011EBB
:1065D00009D0D0230370CA3B4670837087808671D0
:1065E000079804F091FD00232B701721A088FFF776
:1065F00075FCA08801F024FCA08801F0FBFC09B028
:10660000F0BD064B9DE7C0463409FF1FFC65FF1F28
:106610001066FF1FF165FF1FF065FF1F7044FF1F2D
:10662000F8B5070008000E0001F07AFE041E18D02D
:106630002620FFF78DFC051E00D12578062004F0EA
:10664000D3FD041E0DD00021062204F0BDFFD0238F
:106650002370C23B21006770A370A680E8B204F0EB
:1066600053FDF8BDF0B585B001930AAB1B78070068
:1066700002930BAB1B7808000D000092039301F00E
:106680004FFE061E22D0102004F0AEFD041E1DD0C9
:106690001022002104F098FF2620FFF759FC002863
:1066A00000D13078D0232370C13BA370009B210020
:1066B0002372019B67706372029BA580A372039B88
:1066C000C0B2E3720C9BE36004F01EFD05B0F0BDA8
:1066D000F7B50D00019001F023FE071E20D00E201B
:1066E00004F082FD041E1BD02620FFF731FC061E9D
:1066F00000D13E78D0232380C53B0622A370F91D2C
:10670000E01C04F099FF019B2A0063810123DD4016
:106710001A401D40210022736573F0B204F0F4FCAE
:10672000F7BD0000F0B585B0029010000D00170015
:106730000A9E039301F0F4FD041E31D0029B002B4E
:106740002ED1039B02795B0724D512231343042225
:10675000002E08D10B99002905D10C99002902D1EE
:106760000D9900291AD01A430D9B2271002B00D0DD
:10677000C9E0002E00D1CFE0002D00D0CCE0606A4F
:10678000002801D004F0F8FE1C21300004F074FF52
:10679000606205E002239A430E33D7E793432371E7
:1067A000654BBA00D458002C00D1AAE0002E10D0BE
:1067B000236A002B03D11C2004F0A6FD20625E4B4F
:1067C000BA00D358186A002803D01C22310004F004
:1067D00033FF0C9B002B12D0574CBB001D596B6A2A
:1067E000002B03D1162004F08FFD6862BB00E35834
:1067F000586A002803D016220C9904F01DFF0D9B47
:10680000002B11D04C4DBC006659B36A002B03D14C
:10681000142004F079FDB0622B59986A002803D047
:1068200014220D9904F008FF380001F079FD051ECF
:1068300067D0414BBA00D358002B62D01A6A34207B
:10684000002A00D11C389A6A002A01D0143080B284
:106850000B9A002A01D01C3080B25B6A002B01D059
:10686000163080B204F0C0FC041E4AD01822002169
:1068700004F0AAFE2620FFF76BFB0190002801D14F
:106880002B780193D0232370029B200063700A238E
:10689000294EA370039BBD00A371AB59A780196A51
:1068A0001830002905D01C22A06004F0C5FE20008D
:1068B00034307359996A002907D003001422143325
:1068C000E060029304F0B8FE02980B9B002B08D006
:1068D00003001C221C330B992061029304F0ACFED0
:1068E00002987359596A002903D01622606104F096
:1068F000A3FE6B462100187904F006FC3800FFF770
:10690000E3FC05B0F0BD10220D9B0D991B69A0188A
:10691000236204F091FE2CE70B9B002B00D13FE794
:10692000012D00D03CE7606A002801D004F024FE6D
:106930001C210B982AE7C046F865FF1F10B5044CD0
:106940002068002803D004F017FE0023236010BD48
:10695000EC65FF1F0B4B07B51A68002A01D1002018
:106960000EBD6946531C012012780731FFF772FCF7
:106970000028F4D002780123100018401A42EED00B
:10698000EEE7C0460866FF1FF0B51F4F01203B68C9
:1069900087B0002B25D09B78059300F0B3FB00282F
:1069A00021D00A20FFF7D4FA04000B20FFF7D0FA19
:1069B000164B05001E78731E9E413B68F6B2191DEA
:1069C000D878FFF757FB3B682900DA7A0433039243
:1069D0009A7901930292009033002000059A04F006
:1069E000F3FB07B0F0BDFFF7B5FF002805D0062088
:1069F000FFF7AEFA04000720D8E70820FFF7A8FA4F
:106A000004000920D2E7C046EC65FF1FE865FF1FC0
:106A100070B50A4E040033780D00FF2B0DD0042012
:106A200004F0E2FB011E08D0D0230370CE3B45707A
:106A30008370C470307804F067FB70BD8044FF1F22
:106A400070B5040006200D0004F0CEFB011E0AD034
:106A5000D0230370CD3B8370054B44701B68858049
:106A6000187804F051FB002C01D0FFF767FF70BDD0
:106A7000EC65FF1FF8B5264F06003B680D0011249A
:106A8000002B05D10522234B1B78134202D112247F
:106A90002000F8BD204A10241268002AF8D012788D
:106AA000002AF5D0DB0719D52B789A1E012A1AD8AF
:106AB0000C2004F029FC132438600028E8D00023BF
:106AC0000A22437029000670023004F0B5FDFFF77A
:106AD0005BFF041E0AD0FFF731FFD9E700F012FB7D
:106AE0000028E1D1E4E7002BE2D0D0E70B4B1B7884
:106AF000032BCDD11D20FFF72BFA094B188000285E
:106B0000C6D0084B04211878074A04F08DFCBFE773
:106B1000EC65FF1FE965FF1F0866FF1FE865FF1FA3
:106B2000E665FF1F1466FF1F60EA0000F7B50193DA
:106B3000194B14001A78052306000F0012201A4280
:106B400021D0012920D1154B1D68002D1BD002201A
:106B50001F2C18D8002C02D0019B002B13D0104BF7
:106B60001F221E706E1C0021300004F02DFD0199C3
:106B70002200300004F060FD310020002C70002F56
:106B800006D004F099FBFEBD064B12201D68DCE721
:106B900004F022FDF7E7C046E965FF1F0866FF1F06
:106BA0008044FF1F0466FF1FF8B50F4E12243368A0
:106BB000002B17D01B780F3C834213D100250B4FBD
:106BC0000221387804F078FC094B042138781D80C4
:106BD00004F072FC074B28001D8033685C7004F0E1
:106BE0005BFA04002000F8BDEC65FF1F1466FF1F70
:106BF0000066FF1FE665FF1F70B5012823D11B4CFF
:106C00002388002B03D01A4A1578002D07D0194B82
:106C10001B68002B02D01878FFF7C6FF70BD3B2B16
:106C200002D93C3B2380F9E7134E0221307804F06F
:106C300043FCFA222388920002215A43307804F060
:106C400003FC2580EAE70B4B1B68002BE6D00B4BBF
:106C50001B785B07E2D5084B0221187804F02CFC66
:106C60000022024B1A80FFF769FED7E70066FF1F7C
:106C7000E465FF1FEC65FF1F1466FF1FE965FF1F3A
:106C8000F8B51E4D2868002803D004F075FC0023D9
:106C90002B601B4E3068002803D004F06DFC0023ED
:106CA0003360184F05243B7818002040234221D040
:106CB000154800F02BFA3B78234213D0202004F033
:106CC00023FB2860002813D02022002104F07CFC44
:106CD000202004F019FB041E306005D02022002182
:106CE00004F072FC002004E0286804F045FC2C60ED
:106CF0001320F8BD00F00AFAF4E7C0460866FF1F4B
:106D00000466FF1FE965FF1F7444FF1F10B50A4C9E
:106D100023681A1E0ED0002808D10130587004F0E4
:106D2000BBF9002805D02368002B02D00021FFF713
:106D300087FE0122100010BDEC65FF1FF7B5274E3E
:106D4000050033680191181E21D05C78244F012C76
:106D500030D1FFF7FFFD002825D02000FFF7F8F81D
:106D60000400412814D91F4B022118781E4A04F050
:106D70005BFB1E4B3C3C1C80022233685A703B7804
:106D8000002B14D128000199FFF75AFE0120FEBD07
:106D9000FA2292004243002AEED0124B02211878C8
:106DA00004F052FBE8E7FFF7D3F80200F3E7002313
:106DB0003B70EBE73B78002BE8D1032004F014FA9A
:106DC000011E08D0D0230370CC3B4570837033681C
:106DD000187804F099F9FFF7B1FDD7E7EC65FF1FCC
:106DE000E465FF1F1466FF1F60EA00000066FF1FD6
:106DF00010B51749838802008B4220D011D815495D
:106E00008B4217D0144900205B1899B2012907D88A
:106E1000926811785A425341D8B2FFF7F9FD012028
:106E200010BD0E4A00209B1807229BB29A42404197
:106E3000C0B2F5E783681878FFF768FFF0E783686A
:106E400099785A78090218781143FFF777FFE7E736
:106E50000A20000006200000F8DFFFFFAFDFFFFF81
:106E6000014B18707047C0468144FF1F10B5064C97
:106E7000207001F031FA207804F096FA052120788C
:106E800000F052FD10BDC0461466FF1F0BB273B573
:106E90000D00002B00DBC4E0884B187804F024FBC5
:106EA000041E0ED00378912B0FD0A22B00D1A1E0AD
:106EB000834B1878FF2852D0210004F025F90028D0
:106EC0004DD180200002684076BD43780F2B76D0EC
:106ED00013D8052B70D00E2BEAD18088794B9842BD
:106EE0002BD8794B98421BD8784B9842E0D1A368B5
:106EF0001878591CFFF774F838E03E2BD8D1837806
:106F0000032B74D06CD8012B6ED0022BD0D1704BD8
:106F10001B68002B23D05B68002B20D098471EE015
:106F20006C4BC0180C28C3D804F03EF91DC2C21522
:106F30000BC20B0B0B3223C23C00674BC018072857
:106F4000B6D8664B1B68002B09D01B68002B06D0F7
:106F5000200098470AE0A3681878FFF7C7F82000D8
:106F600004F0C2F8ADE7A068FFF762F800289FD0F0
:106F7000F5E7A3681B78002BF1D0554B1B68002B5D
:106F8000EDD01B68002BEAD0210055489847EDE76B
:106F90004F4B1B68002BE2D01B68002BDFD0210079
:106FA0005048F3E7504B1B68002BD8D05B68002B90
:106FB000D5D021004348E9E7FFF7EAF9CFE7808819
:106FC0004A4B984203D04A4B984200D070E7464B58
:106FD0001B68002BC3D05B68002BC0D02100D5E715
:106FE000153B012BBBD963E7FFF798FAB7E7FFF72B
:106FF0007DFAB4E73F4B1B78042B07D100236A4688
:1070000013800179408800F0B5FCA8E7364B1B6877
:10701000002BA4D05B68002BA1D001003648984714
:107020009DE7012421420AD0294B1B68002B04D084
:107030005B68002B01D000209847012043E78B07B5
:107040000AD5264B1B68002B04D05B68002B01D0AF
:1070500020009847022036E70421280008400D420E
:1070600000D131E7254E3388002B21D0013B9BB264
:107070003380002B1AD1FFF7DBF800280AD0204B11
:107080001C70164B1B68002B04D05B68002B01D0D2
:1070900020009847FFF7C6F8694601F0F1FC684602
:1070A000FEF7FEFF1D20FEF753FF308004200AE7A5
:1070B000024B187804F000FAF8E7C0461466FF1F88
:1070C0008144FF1F0E200000012000000910000075
:1070D0000C66FF1FFEDFFFFFAFDFFFFF1066FF1F25
:1070E0000C2000000B200000F465FF1F0D200000A5
:1070F00013200000E965FF1FFFFF0000E665FF1F8A
:10710000E465FF1F10B501F08BF910BD014B18604D
:107110007047C0461066FF1F0B880020162B01D851
:1071200017230420014A13807047C046BE65FF1F25
:1071300000207047074A03001188814207D09188D8
:107140000020994202D101308000101870470020C1
:10715000FAE7C0461C66FF1FF0B58F7806000D00E9
:10716000C7B01E2F15D1FFF7E5FF051E03D1002480
:10717000200047B0F0BD00223B003100C0780092F3
:1071800000F0A2FB0400A81C00F0C3FBFF23EB707F
:10719000EEE7264B062403931B78FF2BE8D0182F2D
:1071A000E6D87B08224A013BDB0002929A589446BB
:1071B000002ADDD0029AD3185B68002BD8D008785B
:1071C000002802D14B78012B02D10624122FCFD1F7
:1071D00007AFAB88697800976446AA68A047041E89
:1071E000C6D1AB78029A5B08013BDB00D3183900AB
:1071F00030005B689847041E0BD1AB78042BB6D0E7
:10720000039A310010782200009700F05DFB040023
:10721000AEE76A78002AABD1AA7805A93B88087145
:1072200030000A704B80FEF747FBA0E78444FF1F45
:10723000B4B800111D4B37B5050098420BD000299A
:107240000AD1FFF777FF002805D11948FFF772FF31
:10725000002800D0058037BD01291AD1FFF76AFF49
:10726000041EF8D001235B420380A378FF2BF2D0E9
:10727000FE2B07D00023E0781422009329001E3350
:1072800000F022FBA01C00F044FB01235B42638062
:10729000E1E70229DFD1013901F0AEF80028DAD1A7
:1072A0002800FFF747FF041EDFD1D4E7FEFF0000F0
:1072B000FFFF0000022210B5074B52421A80074818
:1072C00001325A809A80DA8000F06EFA044801F0A8
:1072D00015F8002010BDC0461C66FF1F5971001133
:1072E000357200110388F7B50400002B02D1022586
:1072F0002800FEBD42680221137825485268FEF737
:10730000A5FD00282ED0234F01253A88002AEFD072
:10731000802321885B0201259B1A9942E8DC0C201E
:1073200003F0F2FF061E31D03B8822889C460023E2
:107330001800019561469DB2491989B2AA421BD82D
:10734000002801D062443A8000233000082208C09F
:10735000210004F071F9104A1368002B13D10025A5
:107360001660C5E76268022113780C485268FEF780
:107370006DFD0028C7D1BAE760681D014019418141
:1073800001330198D6E71A001B68E6E71325AFE73B
:1073900022B900118244FF1F1866FF1F20B9001197
:1073A000014B18707047C0468444FF1F14230A0025
:1073B00010B51A40194204D00122102101F038F80A
:1073C00010BD4B06F9D4012088434000F8E710B502
:1073D00014008B0604D50122102101F029F810BDFC
:1073E00008230A001A40194202D14BB2002B0FDACF
:1073F000102101F01DF8002808D02300F9331B7874
:10740000002BECD0F8342378012BE8D10020E6E7FC
:1074100003208907FAD4E2E7F0B51F00184B85B0C6
:107420001C68019002910392002C27D1200005B026
:10743000F0BDA5683301ED186B89019A934211D311
:10744000029A93420ED8002F04D10A9B002B10D130
:107450002C00EBE73B002978039A6868FEF7F6FCFE
:107460000028F2D10136B6B2A388B342E1D824682D
:10747000DAE7A3680A9A5B891380E9E70026F3E755
:107480001866FF1F37B50C000A884988012391420E
:1074900017D3002A15D0651D23792A0002210A4836
:1074A000FEF7D4FC102300280BD0237961882088B4
:1074B00000242A000094FFF7AFFF0A23A04200D067
:1074C000230018003EBDC04622B9001113B50A00C2
:1074D00008884988012388420BD8002809D0002455
:1074E000137905320094FFF797FF0A23A04200D0DA
:1074F0002300180016BD13B50A0008884988012327
:1075000088420BD8002809D0002413790532009452
:10751000FFF782FF0A23A04200D02300180016BD07
:10752000F0B58BB003904A8808880E000123824290
:1075300055D3002853D00023012704AC2370002228
:10754000718813000092FFF767FF051E3ED0207878
:10755000002835D12B78022B18D167706A898300F7
:107560000130E31880005A8069680222201804F074
:1075700063F823780133DBB22370042B19D93B0065
:107580006889013080B2002BD9D01FE002236370DC
:10759000122358436A89231804305A8069681022DC
:1075A000201804F049F823780133DBB22370002B54
:1075B000E5D10C4A6B899B185A425341DBB2DFE795
:1075C0006378012BE4D12B78022BC7D022780A23D1
:1075D000002A04D021000398FEF798F90023180030
:1075E0000BB0F0BD0100FFFF0F4BF0B504001868B1
:1075F000002816D083685D89A54207D88288AE1816
:10760000B44203DA12019A18934201D10068EFE7FD
:107610001E005F891036A74204D1002900D00D80DA
:107620001800F0BD3300EFE71866FF1F70B50500C6
:107630000C0008880021FFF7D7FF03000120002B72
:1076400004D022002800197AFFF7C1FE70BDF7B5FB
:107650000C00002501902300F6331B78AB4201D8C3
:1076600000200AE06B00E65A00213000E718FFF71F
:10767000BBFF002802D126800130FEBD017A0198AF
:10768000FFF794FE002802D03B882380F5E7013500
:10769000EDB2E0E710B5040008880021FFF7A4FF71
:1076A00003000120002B03D02000197AFFF77EFE93
:1076B00010BD0000054B1B68002B01D1180004E031
:1076C0009A6852898242F6D1988870471866FF1FDF
:1076D000F0B50E27002687B0039302ABFF183E805B
:1076E00005001F4B40891400984207D02B780130C9
:1076F00000976A6880B2FFF78FFE060002212B78A0
:1077000018486A68FEF7A2FB00280FD06C89200099
:10771000FFF7D0FF002802D0013C0419A4B2039B5C
:10772000002B00D01C80300007B0F0BD02212B7868
:107730000D486A68FEF78AFB0028E7D102212B7802
:107740000A486A68FEF782FB002807D0002EDED0C8
:107750003B88A342DBD17489013CDFE76C89DEE71B
:10776000FFFF000022B9001120B900111EB900115D
:1077700070B504000D001600FFF7DCFC002803D0F4
:1077800083781720FE2B05D0002E04D1290020007D
:10779000FEF738F970BD01221021200000F048FEEC
:1077A0000028F3D0F6E70000014B18607047C04690
:1077B0002866FF1F37B56B469D1D0100040002229D
:1077C000280003F0B9FC2B88B02B0ED12379122BA3
:1077D00009D12300FF339B78012B06D1012160885A
:1077E00000F0E0F801E01B2BF8D037BD10B5054BD9
:1077F0000421187000F098F8FFF75CFDFEF780FB9D
:1078000010BDC0462C66FF1F0020F0B50BB20F0064
:1078100087B0834234DA274B187803F065FE051EE3
:107820002BD00378A02B25D103AE3100FEF7F4F85E
:10783000041E0BD1B378DB0724D51F4B06341B681D
:10784000002B03D03100688898470400A8680028FE
:1078500001D003F0C9FE002C08D1184A039B134045
:10786000174A934206D0B3781B2B03D001216888B6
:1078700000F098F8280003F037FC802000027840E0
:1078800007B0F0BD0F4B1B68002B10D0310068888B
:107890009847041EDAD07378002BD7D1B27801A9AB
:1078A0000A704B800C716888FEF706F8CEE7062454
:1078B000F1E7C0462C66FF1F2466FF1F00FFFF0094
:1078C000000112002866FF1FF7B5019082204000DA
:1078D0000D0017001E0003F087FC04001320002C8D
:1078E00012D0B02320002370089BFC2267706580B3
:1078F00026710830002B08D0190003F09DFE2100EE
:10790000019803F001FC0020FEBD089903F05CFE25
:10791000F5E710B5041E06D00078FD2803D803F063
:1079200013FEFF23237010BD0A1F93B210B504008D
:107930000220032B05D882400020024BD1529B1815
:107940009C7010BD4C66FF1F0B8870B5043B040093
:107950000D000220032B0BD80121200000F04CFD6C
:1079600003001420002B03D02900200000F0DEFBD0
:1079700070BD000007B51300034A00920A00012100
:1079800000F02CFC0EBDC046B17B001107B5019282
:1079900003220092024B0A00122100F049FC0EBDA6
:1079A0002F7C001107B56B4601AA11800449D880CD
:1079B00008780633012802D1190003F075FC07BDD1
:1079C0002D66FF1F0C4B10B518700023FF210B4ACA
:1079D0001380138193819380094A538013705172ED
:1079E00093819372D174D3821375517703F0F4FCB1
:1079F00000F0FCF910BDC0465C66FF1F4C66FF1F1F
:107A00002E66FF1FF0B58DB06B46002003910C224F
:107A10009B5E834200DBB0E05D4B187803F064FDB1
:107A2000051E00D1A4E00378902B00D09DE006AFA6
:107A300001004688380000F013FA79680400002934
:107A400000D19CE03B88052B6ED13B89032B1CD9D0
:107A500005AC200000F0A2F86288172A61D83989A5
:107A6000131D994231D17968237804310291D907E5
:107A700038D5607800F08EF9071E06D00023037118
:107A80002378012B08D0132B23D0A868002800D11D
:107A900078E003F0A9FD75E06288029909A800F07A
:107AA000A6F80290380000F08BF909AA2378387AFA
:107AB0000192002231000092029A00F012F938007F
:107AC00000F064F9029B002BDFD0300000F080F959
:107AD000DBE70378032BD8D16288029909A800F06C
:107AE000D6F8DEE7122B13D1029909A800F0B5F8F9
:107AF000021EEAD127498B88002BC6D0887909A9B4
:107B00002378019161780091310000F0EAF8BCE738
:107B1000002302AA93833000617809AAFFF72AFFA5
:107B2000B3E71D4B0993F6E7042B02D09A1F012AF5
:107B3000ABD8184A043B9B00995A0029A5D0D2180B
:107B4000907831003A0000F0AEF800289DD13B88D3
:107B5000042B03D001213000FFF724FF012C04D1B6
:107B6000A868002801D003F03FFD280003F0BCFA0C
:107B70008020039B0002434018000DB0F0BD012897
:107B800000D182E701213000FFF70CFFEDE7C0468E
:107B90005C66FF1F4C66FF1F010017000B78037027
:107BA0004B784370CB788A781B021343438070472D
:107BB0000A88030002700A88120A42700A88012AA1
:107BC00006D14A8882704A88120AC270042070471F
:107BD00002208242FBD14A8804309A704A88120AF5
:107BE000DA708A881A718A88120A5A71EFE710B51A
:107BF0000400012082420CD94B780A781B021343FF
:107C00002380834206D1CB788A781B02134363809A
:107C1000002010BD022BFBD1CB788A781B021343C6
:107C200063804B790A791B021343A380F0E70B882A
:107C300003700B881B0A43704B8883704B881B0AA8
:107C4000C3708B8803718B881B0A4371CB88837147
:107C5000CB881B0AC3710820704703000120082A43
:107C600014D14A780878120202431A80CA788878B8
:107C7000120202435A804A790879120202439A801A
:107C8000CA798879120202430020DA80704710B561
:107C900004000120022A05D100204B780A781B023B
:107CA0001343238010BDF8B5060010200F00150007
:107CB00003F09AFA04000120002C0ED0A0230C221D
:107CC000290023806780201D002D07D003F0B4FC1D
:107CD0002100300003F018FA0020F8BD03F074FC16
:107CE000F6E7F7B51E00009008AB142017001D78CA
:107CF000019103F079FA041E12D0A2230370019BB4
:107D000047704380099B057146710C220830002B97
:107D100007D0190003F090FC2100009803F0F4F95B
:107D2000F7BD099903F050FCF6E737B5041E0FD0F4
:107D30004388002B0CD00025C1881323007A17221A
:107D400001950095FFF7CDFFFF23658063722570D5
:107D500037BD000010B50C4904004A88002A09D03C
:107D60008B89002B05D00020CB8A0222834201D0D0
:107D700010BD012213000A20434300204032C854A2
:107D8000C81842800472F3E72E66FF1F0023438069
:107D900003707047094B00211A0010B55C88002C55
:107DA00006D01C79844203D10A234B43D01810BD5E
:107DB00001310A330329F1D10020F8E72E66FF1FB5
:107DC00010B50400407A03F0BFFBFF23637210BDBF
:107DD0007047043010B580B203F01EFC002803D0B9
:107DE0000421494203F0B0FA10BD000070B500252F
:107DF000104CA0682580A581A580A84202D003F080
:107E0000F3FBA56000250C4C0C4B606D1D8023001E
:107E100058331D70A84202D003F0E6FB65650025CB
:107E20006068002801D003F0DFFB013508340A2D1B
:107E3000F6D170BDF466FF1F9866FF1FE866FF1F4E
:107E400070B5041E09D1054D2880A881A880A868B6
:107E5000002802D003F0C8FBAC6070BDF466FF1FC1
:107E6000F0B54B8885B00193002343600A79050083
:107E70000F00022A00D07BE0CA88032A17D98B683A
:107E80005E7819783602DC78D8790E4399781B7AB7
:107E900024021B020C43034353495BBA0B80331D7E
:107EA00093421ED1042C04D0631F022B0ED9012053
:107EB00015E0019A4D4B1201D35A002B06D00198C0
:107EC000FFF7BEFF4A4A1369013313610421B86802
:107ED0002E812C80494203F037FA6860002005B0FB
:107EE000F0BD434D042C06D0631F022B0FD9EB6865
:107EF0000133EB60DBE7019A3C4B1201D35A002BB4
:107F000005D00198FFF79CFF2B6901332B61374B9C
:107F100030000293019B029A1B01019300230199F7
:107F20008C468B52130063449C8003939E81FFF721
:107F300050FF039B041E986016D00421B868494284
:107F400003F002FAFA880100043A200003F074FBFF
:107F50000199029AFB888A5A043B9B18029A8B5219
:107F60002B6801332B60A2E7AB690133AB619EE75D
:107F70001E4B0293019B1E01029BF35A002B2DD036
:107F800002998C19A068002828D0012A26D1FA88E5
:107F90009B189BB27352A189994217D39B1AC018A0
:107FA000B96803F049FB029BA289F35A934200D0BF
:107FB0007DE700222B81A3882B80A3686B60029B46
:107FC000F2520B4A53680133536070E7084A9368D2
:107FD000013393600198FFF733FF68E7044A536960
:107FE00001335361F6E7C0465E66FF1FF466FF1F6C
:107FF0006466FF1F70B5051E15D10B4C0B4B188026
:10800000230058331870606D002802D003F0ECFA9A
:108010006565250050356068002801D003F0E4FA5A
:108020000834AC42F7D170BD9866FF1FE866FF1FA9
:10803000F0B51700A12285B0920001934243394B5D
:1080400006001B680C009B18D933FF331D78FDF721
:1080500051FF0430854204DD3000FDF74BFF043052
:10806000C5B2BD4207D33A0000213000019B03F0A6
:108070007BFA05B0F0BD2900380003F0DDF82300DD
:10808000C6B250331E700393019B2900636538000C
:1080900003F0EAF8CBB20293002B02D0039B013627
:1080A0001E7000262300503303931B78B34204D87C
:1080B000606D002831D10020DBE7029A2800002AF9
:1080C00004D0013B1000B34200D02800F700E719AC
:1080D000387002F0A9FF786000280ED03A78019934
:1080E00003F0AAFA019A3B780136D3180E4A01939D
:1080F000D369F6B20133D361D4E7039B187060658E
:10810000A74205D1084A1320D36A0133D362B0E7EE
:10811000606803F069FA0834F2E703F065FA0023B7
:108120006365C8E73409FF1F6466FF1FF7B50D00DC
:1081300007000421686803F007F92B890400037025
:108140002B891B0A43702B8883702B881B0AC370F2
:108150002E8902250436F6B2FB2E15D81B4B9F4202
:1081600014D10C2003F040F81135011E0CD09023DF
:1081700003708E3B0371043B4380154B8460C680C3
:10818000187802F0C1FF00252800FEBD5C237B4368
:10819000104AD3180093583301931B78002B0FD14A
:1081A0000300320038000099FFF742FF019B0500F1
:1081B0001B78002BE8D13800009903F04DF9E3E774
:1081C000054A0725536A01335362DDE7FEFF0000CD
:1081D0005C66FF1F9866FF1F6466FF1FF0B587B0DF
:1081E000009017200F0016000193FFF7F2FD1325F2
:1081F000041E19D00C98031E02D00199201D984727
:10820000030AE370052302AAA0700430908127704E
:108210000098667003A993800494FFF787FF051EFA
:1082200002D0200003F0E0F9280007B0F0BD000004
:10823000F0B587B01F000CAB1B78039105930121AB
:108240000DAB06001C78049200F0D6F81425002827
:1082500021D02000FFF77EFD0135041E1BD01149FF
:10826000059B0A7803700132D2B2131EC68001D179
:1082700001231A000B7022713000049B03990097B0
:10828000FFF7ACFF051E09D1230021000648074A6D
:10829000093302F031FF280007B0F0BD00236380EE
:1082A0002370F8E76066FF1F2B7D0011307500001A
:1082B000F8B505000E00064C064F2368002B02D0CF
:1082C0003100280098470434BC42F6D1F8BDC046BE
:1082D0000467FF1F1867FF1F0123064A5B42538094
:1082E000002313715362044A136053609360D36098
:1082F000136170471867FF1F0467FF1F0200002308
:1083000010B506499C000859002801D1625010BDE3
:108310000133052BF6D11320F9E7C0460467FF1F90
:10832000034A5388181A434258414042104070474C
:108330001867FF1FF0B585B002930AAB1F780CAB2E
:108340001B88009008000E0001920393FFF7E8FFDE
:1083500005001120002D1BD10E48FFF7E1FF04009E
:108360001520002C14D006220B99A771E01D03F0F4
:1083700063F9019B30002371029B29006371009B0C
:1083800066802370039B6562E381FFF791FF2800FD
:1083900005B0F0BDFFFF000010B5FFF7C1FF0400FE
:1083A0000220002C12D060880121FFF781FF606A53
:1083B000002801D003F0E0F828220021200003F07B
:1083C00003F9012300205B426380207110BD00008F
:1083D00030B5074A074C5588010013780020A542A4
:1083E00004D05B1A59424B415842104030BDC04640
:1083F0001867FF1FFFFF0000084A10B501230C009B
:10840000904208D0FFF78CFF031E04D0037923406D
:108410005A1E9341DBB2180010BDC046FEFF00009B
:10842000024B1879431E9841C0B270471867FF1F6E
:1084300070B504000D001600FFF772FF002804D18C
:108440000D4B9C4200D0143070BD416A0379052069
:10845000002907D012221A40102A02D10520002E2E
:10846000F2D10F20DB06EFD5897E0C20A94289418D
:10847000494249420840E7E7FEFF0000030010B50B
:10848000002800D110BD0348034A41889142F9D029
:108490009847F7E71867FF1FFFFF0000002330B57C
:1084A000C45CCD5C6C40D4540133102BF8D130BD8A
:1084B0000F23002210B5C45C64002243CA54C25C7E
:1084C000D209013BF7D210BD0200010010B52032E5
:1084D000103102F081FE10BDF0B58BB0039010207A
:1084E00005931700049102F00FFF0090102002F096
:1084F0000BFF009B13240190002B05D000280CD10A
:108500001324009803F038F8019B002B02D01800C8
:1085100003F032F820000BB0F0BD102002F0F4FEA2
:108520000600102002F0F0FE13240500002E00D1FA
:10853000AEE0002819D01022002103F045F83200E7
:108540002900039802F048FE041E0ED133787F2BD9
:1085500051D830000099FFF7ABFF009B1B787F2BB1
:1085600053D801990098FFF7A3FF300003F004F8F7
:10857000002D02D0280002F0FFFF002CC1D11020F6
:1085800002F0C2FE0600102002F0BEFE0290002E95
:108590007CD0002878D03A000F3223000125121138
:1085A00005D00F333B4015B25A4253411BB26A1EED
:1085B0001201002B33D0049BD2B298180099029A72
:1085C000FFF76CFF013D10220021300002F0FCFF9C
:1085D000ADB2049F2D017D19AF4242D0002C33D0A3
:1085E000300002F0C9FF029B002B00D189E7180080
:1085F00002F0C2FF85E729003000FFF759FF28008D
:108600002549009AFFF74AFFA7E729000098FFF7DE
:108610004FFF28002049019AFFF740FFA5E70F21EF
:108620000F4004998A18D9B28F4208D9D15C06A8A4
:1086300019540133102BF6D1029A0199C0E7791A27
:1086400048424141C901F2E73900300006AAFFF76C
:1086500025FF3200039806A902F0BEFD1037040082
:10866000BAE7002CBCD13000029906AAFFF716FF2A
:10867000320006A9039802F0AFFD08220400310081
:10868000059802F0D9FFABE71324A9E71324AAE762
:10869000002800D06EE733E728B90011F0B58BB0A1
:1086A0000F0016000225009000283FD0002A3DD080
:1086B0000B1DDBB21800029302F026FE1135041EDA
:1086C00034D0FDF757FD05003A000099201D02F057
:1086D00043FFEBB20393E3702B0CDBB22F0A009342
:1086E0006370FFB22B0E2370A7700193FDF73CFD62
:1086F0001022010006A802F02FFF2100029A04AB0D
:1087000006A8FFF7E9FE051E0DD1039B0822337072
:10871000009B04A9B370019B7770F370301D02F0C9
:108720001BFFFDF72DFD200002F026FF28000BB0F7
:10873000F0BDF0B58FB00D00149E03900492059328
:10874000002A03D1022420000FB0F0BD002EF9D082
:108750000398FFF7E5FD1424071EF4D072783378F0
:1087600012021A43B3781B041343F27812061A4319
:10877000036A0192934201D30133E3D1002D03D068
:108780003B7901249B07DED50822002106A802F0D0
:108790001BFF059B13240433DBB21800029302F085
:1087A000B3FD051ECFD0059A0499043002F0D4FE23
:1087B00004223100280002F0CFFE390010221031CF
:1087C0000AA802F0C9FE2900029A06AB0AA8FFF720
:1087D00083FE041E0FD1082206A908A802F0BCFEE1
:1087E0000822311D08A802F0FFFD012807D10199D8
:1087F0000398FDF7D9FC280002F0BEFEA3E7012490
:10880000F9E7000070B51C4C05002368181E10D055
:10881000002D14D11A78002A0CD1981C083202F0CD
:108820000BFF02F0E9FE0135002808D123681D7016
:10883000012070BD0A331800082202F0FDFE2368F3
:10884000002BF5D0122002F0CFFC061E0DD0C12364
:1088500021680370457002311022023002F0ECFEF4
:1088600023683100587802F04FFC206802F084FE43
:1088700000232360DCE7C0464067FF1FF8B5040013
:108880002020FDF765FB0D4EA700BB590500002B0E
:108890000DD000280BD0D878FF2809D108492A002C
:1088A0000C55F35907480333611802F025FCF8BD55
:1088B000290002F081FE0028F0D1F8E75C67FF1F75
:1088C0004467FF1FD59A001170B5064D84006359A7
:1088D000002B05D0D87802F037FEFF226359DA70FA
:1088E00070BDC0465C67FF1F70B506008CB00C0001
:1088F000150000213022684602F066FE3100102289
:10890000684602F029FE1D2021000322684402F07F
:1089100023FE6846FFF7D8FD2D210400032228001E
:10892000694402F019FE20000CB070BDF0B50700DC
:10893000160097B001931CAB1D7830221EAB00913E
:108940000AA800211C7802F03FFE102239000AA874
:1089500002F002FE1022002102A802F035FE0722DA
:10896000310002A802F0F8FD072202AB9818631E3E
:108970009C41019902F0F0FD02AB9C732B005A1E42
:10898000934102AAD3730021102206A802F01CFE14
:1089900006221D9907A802F0DFFD1A2002ABC018BD
:1089A00006221F9902F0D8FD102200990EA802F0AD
:1089B000D3FD102202AB0EA908781C78013A604062
:1089C000D2B2087001330131002AF5D10AA8FFF7AD
:1089D0007BFD102212A904000EA802F02DFE102229
:1089E00006AB0EA908781D78013A6840D2B208702B
:1089F00001330131002AF5D10AA8FFF765FD0443D0
:108A000010222098E4B212A902F0A6FD200017B0AF
:108A1000F0BD70B50E0014008CB001001022684645
:108A20001D0002F099FD3100082204A802F094FD17
:108A30002100082206A802F08FFD6846FFF744FDDA
:108A400004001022280008A902F086FD20000CB0C6
:108A500070BDF8B506000D0000243719AC4200D3F4
:108A6000F8BD02F009FC030A3B70631CDBB201375E
:108A70009D4203D90234F054E4B2EEE71C00EDE766
:108A800073B506000C000225002819D0002917D064
:108A9000032101A8FFF7DDFF6B469A793F231A40B7
:108AA000013313436A463000937101A92200FFF796
:108AB0001BFF051E04D10322E01C01A902F0BCFD2E
:108AC000280076BD03785807DA08C00FD20080006E
:108AD0009B0710439B0F1843C0B2704707230B40FE
:108AE000C908C9000B4303707047000070B504004B
:108AF000FFF7EAFE134DA4006359002B21D0186A3A
:108B0000002801D002F038FD2B59986E002801D0C2
:108B100002F032FD2B59D86E002801D002F02CFD56
:108B20002B59186F002801D002F026FD2B59586FE1
:108B3000002801D002F020FD285902F01DFD00237D
:108B40002B5170BD5C67FF1F0E4B8000C35870B582
:108B50000C00002B0FD09D68002D0CD02B78201D11
:108B60000B706B784B70A97CFFF7B8FF2B7E2372DC
:108B70006B69E36070BD10220021200002F024FD2B
:108B8000F8E7C0465C67FF1F014B18607047C0469E
:108B90005867FF1F074A03008000825810B5002A5B
:108BA00006D0D088984203D1012901D1FFF79EFF5A
:108BB00010BDC0465C67FF1FF0B5264E95B087001C
:108BC0000B93BB590500099112200A92002B31D05A
:108BD000D888FFF7A5FB04001420002C2AD0280019
:108BE00010A9FFF7B1FFBB591E781D6A002E23D0D4
:108BF0000895FDF7FFFA07000020FDF701FB07903D
:108C0000A379E61D069310AD0CA9089800F0E2FACE
:108C10000EA9280000F0D7FA0B9B0A990493069B33
:108C200009980293079B0396019300970EAB0CAA39
:108C3000FFF77CFE15B0F0BDFDF7DCFA06903000C2
:108C4000FDF7DEFAE31DA779079310AB0600089342
:108C5000DAE7C0465C67FF1F30B50C4C85002A5927
:108C6000030085B00120002A0ED018006946FFF7E6
:108C70006BFF2B591A78D888054B002A00D1054B79
:108C80006A46072100F0D9FB05B030BD5C67FF1FC5
:108C9000C7910011D591001130B5094C85002959B3
:108CA00085B010226846253102F0C6FC2A591121F0
:108CB000044BD0886A4600F0C0FB05B030BDC0460A
:108CC0005C67FF1F7192001130B5094C850029596E
:108CD00085B010226846353102F0AEFC2A591121C8
:108CE000044BD0886A4600F0A8FB05B030BDC046F2
:108CF0005C67FF1FAF920011F7B54D4F8600102043
:108D0000F4590D0002F000FBF3592062186A132297
:108D100000286CD0033A29009C6802F08DFCF359BE
:108D20001A780192002A58D11E6A227D317B94461E
:108D300051400122019F114201D167461740217D18
:108D4000914339432175377B4F40BC46604600272D
:108D5000800701D44F081740012102208F40227D57
:108D600082433A432275377B5740BC466046002712
:108D7000400701D497080F400420227DBF008243A2
:108D80003A432275627D002794466046727B4240DA
:108D90000A4201D167460F400121627D8A433A436E
:108DA0006275777B5740BC4660460027800701D438
:108DB00057080F400220627D7F008243174367758A
:108DC000767B00227E40760701D4BA080A4004264A
:108DD000617D9200B1430A4362756A78002A08D027
:108DE0006278002A05D005220533DA7700221000C8
:108DF000FEBD04222979114205D1A17C114202D184
:108E00000533033AF1E7019A21782C78002A02D140
:108E10000A002100140018220429E8D8042CE6D8FE
:108E200005206043034A05331218525CDDE7C04653
:108E30005C67FF1F38B9001110B50A001121024B01
:108E400000F0FBFA10BDC0460B9300110B0030B5CB
:108E500087B001AD2B806B4604001100981D0822DD
:108E600002F0EAFB2A000B212000024B00F0E5FA99
:108E700007B030BD3393001110B50A001121024B29
:108E800000F0DBFA10BDC0468793001113B50B004C
:108E900011006A4613706B4604000622581C02F04B
:108EA000CBFB6A4608212000014B00F0C6FA13BD37
:108EB000A793001110B50A001121024B00F0BDFA72
:108EC00010BDC046F79300117FB505000B4BAA00FB
:108ED000D4580800002C0FD0666F237FE2882178D9
:108EE0000396266F0296E66E0196A46E0094FDF737
:108EF00019FC2800FFF7FAFD7FBDC0465C67FF1F25
:108F000010B51721FFF7E0FF10BD000070B50A0093
:108F10000D00064B0221040000F08FFA06002978AC
:108F20002000FFF7D1FF300070BDC046D79200117E
:108F300070B586B000236A461370836804001D78FC
:108F4000681E0A2859D801A902F09EF9060633378F
:108F50003B3F43474B4F5300180000F042F90623B4
:108F600012284BD000281BD16088FFF7D9F90823BD
:108F7000002813D04279002A47D1264B1A780723BC
:108F800012070BD5244B1A680723002A06D016684F
:108F9000002E03D0290001AAB04703006A461370CF
:108FA0006B461B786088002B2AD1FFF767FC06B060
:108FB00070BD180000F06CF9D4E7180000F087F9D4
:108FC000D0E7180000F093F9CCE7180000F0ADF9F5
:108FD000C8E7180000F0C3F9C4E7180000F0F6F97C
:108FE000C0E7180000F0F6F9BCE7180000F013FA2B
:108FF000B8E7180000F013FAB4E707236A461370C5
:1090000069466088FFF782FFD1E70523012AC5D1B1
:10901000024BB8E7E965FF1F5467FF1F5867FF1F42
:10902000F8B52C4F8600F35904000D00002B40D0FA
:10903000DA8882423DD15A78062A33D11A78002A3A
:109040002ED0012099681A6A097D014206D0157B4D
:10905000054203D007225A700120F8BD02200142C8
:1090600004D0157B054201D00922F4E70420014217
:1090700004D0127B024201D00B22ECE7164B1B6896
:10908000002BE9D05B68002BE6D020009847BB5945
:1090900000215B78122BDFD12000FFF715FFDBE703
:1090A0000E4BECE7112A04D1002900D0322529000B
:1090B000F2E7002D08D12000FFF732F9002803D095
:1090C000102302791343037121002800FDF7A8FA49
:1090D000C2E7C0465C67FF1F5467FF1F5867FF1F4A
:1090E00070B50E4E8500AB590400002B13D01B78D1
:1090F000002B11D10A4B1B68002B04D05B68002B9E
:1091000001D02000984773595B78122B03D10021BE
:109110002000FFF7D9FE70BD024BECE75C67FF1F34
:109120005867FF1F5467FF1F094B8000C35810206A
:10913000002B0CD01A6A002A09D09B68002B06D09D
:10914000127A1B7E101C9A4200D9181CC0B27047BC
:109150005C67FF1F70B503000D0014000220002A99
:1091600030D000292ED013700B78081D53704B7827
:109170009370FFF7A7FCE070012002212B7A237186
:109180006B7B034063716A7B0A4013430422637163
:109190006E7B1640334363716E7BF608F6003343F3
:1091A00063712B7B0340A371287B014000200B439C
:1091B000A371297B0A401343A3712A7BD208D200F2
:1091C0001343A37170BD10B50A0001000120FFF721
:1091D000C1FF10BD10B50A0001000220FFF7BAFF61
:1091E00010BD70B506000C000220002E30D0002902
:1091F0002ED07378201D0B70B3784B70F178FFF789
:109200006DFC01223579257271794B1008001340ED
:10921000934010400343881010408000C908034366
:10922000C9000B436373B1794B100800134093409E
:1092300010400343881002409200C9081343C9003C
:109240000B4321202373FCF783FE854201D21220B9
:1092500070BD2220257AFCF77BFE8542F7D8237863
:109260001820042BF4D86378012BF1D80020EFE705
:10927000030010B50220002909D0002B07D00322DB
:10928000481C0A7019000D3202F0D6F9002010BDFA
:1092900003000222080010B5002B06D0002904D0DC
:1092A0000E32591C02F0C8F90022100010BD030054
:1092B00010B50220002909D0002B07D00422481C39
:1092C0000A7019000C3202F0B7F9002010BD10B579
:1092D000FFF7DEFF10BD03000220002906D0002B9F
:1092E00004D0052200200A701B784B7070470300E1
:1092F0000220002B08D0002906D05B7800200B70DC
:10930000013B082B00D918307047030010B502202C
:10931000002909D0002B07D00622481C0A7019002A
:109320000A3202F089F9002010BD10B5FFF7B0FF36
:1093300010BD02000B00022010B500290ED0002A3B
:109340000CD007211970118859701188090A997079
:1093500011180822D81C02F06FF9002010BD03007C
:109360000A00022010B5002B0CD000290AD09978F1
:109370005878090201431180901CD91C082202F080
:109380005BF9002010BD030010B50220002909D0B0
:10939000002B07D00822481C0A701900921802F00E
:1093A0004BF9002010BD02000B00022010B500296F
:1093B0000BD0002A09D0092119701178181859709A
:1093C000511C062202F038F9002010BD10B5FFF73D
:1093D0005FFF10BD02000B00022010B5002A09D06B
:1093E000002907D05178197011180622581C02F074
:1093F00023F9002010BD030010B50220002909D078
:10940000002B07D00A22481C0A701900063202F00D
:1094100013F9002010BD10B5FFF73AFF10BD020090
:109420000B00022010B5002A06D0002904D0180035
:109430005178FFF753FB002010BDF0B585B0170041
:109440001E006A4606230500080091819380FEF7FE
:10945000C0FC1324011E02900CD03800B047041E3B
:1094600005D1280001A9FEF76FFA041E02D0029868
:1094700002F0BAF82800FFF701FA200005B0F0BDAD
:10948000F0B504008BB0019115000021102202A854
:1094900002F09AF8334EA700B85900283CD0C38890
:1094A000A34239D10378002B36D14278062A18D14D
:1094B00002000100553235310C3006ABFFF7A9FA36
:1094C000002829D12000FFF72FFE020006A902A8DC
:1094D00002F0B2F8200002A901F00EFF01200BB04B
:1094E000F0BD816E002917D00B8A112A28D19D4228
:1094F0000ED101981231093A01F076FF012807D107
:10950000BB5920009D6EFFF70FFE29000200DEE729
:1095100032212000FFF7D8FC2000FEF701FF061ED5
:109520001BD0416A002918D00B8AAB4215D1082202
:109530000198123101F058FF01280ED1716A0AE03A
:109540009D42E9D108220198123101F04DFF012816
:10955000E2D1BB59996E8A7EB9E7200001F0CCFFB9
:10956000BCE7C0465C67FF1FF0B56B4D87007E59B6
:1095700085B0337802900393002B00D087E0B36866
:10958000346A01937078062817D101221B7D13429B
:1095900002D0217B114218D10222134202D0217B3A
:1095A000114251D10422134203D0237B134200D035
:1095B0008BE0019B5A7DEB5991E007380428F8D8DD
:1095C00001F062FE032E42678300B36E002B03D1CD
:1095D0001C2001F099FEB066EB599C6E002C1CD04B
:1095E00010220021200001F0EFFF0298FFF79CFD00
:1095F00001002000FFF72DFA01F03EFE208220003E
:1096000008211230FFF725FA0298FFF78DFDA076AA
:10961000EB592100D888FFF70FFC0822EB591CE01A
:10962000B36E002B05D01A00198AF0881232FFF7AA
:109630000DFC0222019B197DEB5911423DD0207B8C
:1096400010423AD0073208E0F488FCF7EBFD010045
:109650002000FFF711FC0A22EB595A70029B9C0074
:109660002A595378073B042B11D8D088FEF758FEAF
:1096700000284ED0C3895A08D2182849029B029864
:10968000CB542B5941180433254801F035FD05B062
:10969000F0BDFCF7AFFD03000120834201D10020A3
:1096A0000393EB59DE88FCF7ABFD03990200300011
:1096B000FFF7ECFB019AEB59117D042211420CD00B
:1096C000217B114209D00B22C7E7F688FCF74CFD3D
:1096D00001003000FFF7EEFB6BE7019A527D01219C
:1096E0000A4204D0607B084201D00C22B5E7022177
:1096F0000A4204D0607B084201D00E22ADE704216B
:109700000A4204D0627B0A4201D01022A5E712224D
:10971000A3E7FA225200B0E75C67FF1F6067FF1FF4
:10972000DF9A001110B5064B1A7804231000184078
:109730001A4200D00348FFF727FA002010BDC046A8
:10974000E965FF1F8844FF1F70B50400FFF7D4FAD6
:10975000051E43D12000FFF77FFA234EA400A05935
:109760008268937CDB0708D50321036A1B790B40D1
:10977000012B02D1017F0B430377431DD97F8B1E41
:10978000022B0DD8022900D00121C088FCF7A0FFD0
:10979000042133591A7F59700A431A77280070BD83
:1097A00001290CD102231022437000210C3001F05A
:1097B0000BFF305910213530FFF74BF9EEE7052943
:1097C000ECD10223D118437010220C3001F034FF89
:1097D00004233259117F0B431377EAE70825182831
:1097E000DCD1053DDAE7C0465C67FF1FF0B58BB002
:1097F000059143887E4F9E00F45915000493002C78
:1098000015D1012902D000200BB0F0BD101D5778F2
:109810001678FFF757F9EB68320002932B7A049918
:10982000019300903B002000FCF71CFFEBE7E3886E
:10983000049A934201D00820E6E72378012B00D157
:10984000D4E0059B581E092800D9CFE001F01CFD8B
:1098500005CE0A29CC506C859AB229000498FFF7EE
:1098600073FFD1E7200029001022453001F0E4FE0B
:10987000B9594B78042B02D1013B4B70C3E70B0065
:109880000A00253335320C310498FFF795F9049816
:10989000FFF702FA0522431E9841BB59C0005A70D7
:1098A000B2E7200029001022553001F0C5FE049BCC
:1098B0004F4C9D00295904980A0006AB55320C31D3
:1098C000FFF77AF929591022453106A801F08CFDDD
:1098D000012808D10498FFF7F7F90590002804D172
:1098E00006222B595A7005988EE708230593FAE74C
:1098F00063780C2B7AD1E36E002B03D11C2001F08E
:1099000003FDE066BB59D86E00286FD010222900F5
:1099100001F092FEBB590498DC6EFFF705FC0D22A6
:10992000A076BB595A706EE7E06E00285ED063786F
:109930000D2B5BD12B8808220382A91C123001F069
:109940007BFEBB599A68517D0222114226D0186ACB
:10995000407B104222D00C32E4E763780E2B45D1D5
:10996000236F002B03D1162001F0CEFC2067BB59DA
:10997000186F002803D01022290001F05DFE0F228D
:10998000BB59CFE763780F2B30D1206F0622691CBB
:10999000103001F051FEBB599A68517D04221142EA
:1099A00003D0196A497B1142D5D100210498FFF7F1
:1099B0008BFA28E7636F002B0DD0BB59586F002836
:1099C000F3D01022290001F037FE0122BB59524288
:1099D0005B6F1A61E9E7142001F096FCBB596067E0
:1099E0005B6F002BE9D126E72978DFE707200BE73B
:1099F0005C67FF1F10B5064C207001F02DFB06219F
:109A00002078FDF791FF0348FEF778FC10BDC046B3
:109A10006F67FF1F958B001100200BB270B50D0012
:109A2000834216DA264B187801F05EFD041E0DD035
:109A30000378922B0ED0A02B37D0224B1878FF281A
:109A40003AD0210001F060FB002835D180200002CF
:109A5000684070BD43780E2B0BD03E2BEDD1837840
:109A6000052B12D0082BE8D181798088FFF7D8FA2E
:109A700008E0154B82889A42DFD183681878591C18
:109A8000FEF7C0FE002817D1D7E7104B1B785B0705
:109A900012D50F4B1B68002B0ED09B68002B0BD0F0
:109AA000C289811D80889847ECE7FFF741FAA068DA
:109AB000002801D001F098FD200001F015FBC5E75A
:109AC0006F67FF1F8144FF1F18200000E965FF1F1B
:109AD0005867FF1F10B50078FFF712FA10BD10B5D8
:109AE0000078FFF7FDFA10BD0C234343084A10B578
:109AF0009B185A68002A03D0012901D1904710BD54
:109B00009B68002BFBD00029F9D19847F7E7C046A6
:109B10008C67FF1F10B5162813D801238340094A0C
:109B2000946B1C439463506B98435063D46B200038
:109B30009843012901D120001843D063116B0B43D6
:109B4000136310BD00800040F0B500240127154BC1
:109B500085B0DA6B144E03921A6C0192DA64019BA1
:109B6000E3403B4217D0039DE5403D400295E5B2FE
:109B700002992800FFF7B8FF316A736A002908D0FC
:109B80003900002B01D0029979402800FFF7C2FF6D
:109B900001E0002BF9D101340C36172CDFD105B0D0
:109BA000F0BDC046008000407067FF1F10B5012463
:109BB00002002000162A08D8054B5968D1402142DE
:109BC00004D01868D0400123184010BD186DF9E783
:109BD00000800040162807D80122064B8240002949
:109BE00003D0D9680A43DA607047D9689143D960D5
:109BF000FAE7C0460038004030B5162818D80324CC
:109C000044430F4BE25C1B199C785D7801232D1BAC
:109C10000135AB40013BA340A140DB430C001228BF
:109C200007D8084992005218116819402143116061
:109C300030BD054A11680B4023431360F8E7C04666
:109C40007FB9001108F0004014F00040C21F70B549
:109C5000D4B20623092C0BD80125084C95400029C5
:109C600008D00021FFF7C8FF23682B43236000239F
:109C7000180070BD2368AB43F8E7C04600380040C9
:109C8000F0B5162826D8214B1B185B78022B21D162
:109C9000032444431E4A1F4EA35C121994780122E8
:109CA00015008540B76B013CE4B23D43A240B5636B
:109CB000194C122815D89B0000290CD117495B18A4
:109CC00099680A439A600123205C154A8340116811
:109CD0000B431360F0BD11495B189968914399607B
:109CE000F1E70E4B00290DD159690A435A61225CF4
:109CF0001328E8D00123203A93400A490868034317
:109D00000B60E7E7596991435961F0E77067FF1FFE
:109D10007FB9001100800040C4B9001100F000407C
:109D2000A0F00040A4F00040F8B500241B4E1C4DEC
:109D30001C4B1B5D012B1FD1184A9269E2401A424D
:109D40000BD00122AA5693402200143AD2B2022A22
:109D500009D815494A6913434B6101340C36023561
:109D6000172CE5D1F8BD0022AA560F4992005218CF
:109D700091680B439360F0E7022BEED1E7B2380015
:109D8000FFF714FF01235840C1B23800FFF778FFF6
:109D90003800FFF70BFF7077DFE7C0467067FF1FE3
:109DA00051B900117167FF1F00F000400122023815
:109DB0008240054B002903D059690A435A61704714
:109DC000596991435961FAE70038004070B50400C1
:109DD0000D000520162C1AD800212000FFF7FAFEEE
:109DE000A31E012B03D801212000FFF7DFFF002174
:109DF0002000FFF72BFF01220A49A2400A4B4868C6
:109E0000012D05D102431B194A605D70002070BD11
:109E10009043486002211C196170996991439961CE
:109E2000F4E7C046008000407067FF1F10B5162899
:109E30000AD80122074B8240002906D019680A433C
:109E40001A600121FFF7C2FF10BD19689143196024
:109E5000F7E7C0460080004070B505000520162DCC
:109E600017D80C2300246B430A4A21009B181C704E
:109E7000094B28005B195C70FFF7A8FF0123AB407A
:109E8000200006490A681A430A6005490A689A438D
:109E90000A6070BD8C67FF1F7067FF1F3480004031
:109EA0003080004070B504000E00FF2813D0032559
:109EB0000540FFF7D1FF084AA3089B009B183F22EB
:109EC000ED00AA40AE40196820009143314319606B
:109ED0000121FFF77FFE70BD18380040F8B505007E
:109EE0000520162D25D80C246C43124BE41863680A
:109EF000002B03D1A3680D30002B1AD002220127BA
:109F00000D4B00215B195A7028002770FFF75EFF88
:109F100063681E1E08D0A3683E00002B04D02800F2
:109F2000FFF744FE4640F6B228003100FFF7F2FD8D
:109F30000020F8BD8C67FF1F7067FF1FF7B5C420B6
:109F4000FF222B4B80001958002491437F3A0A438B
:109F50001A508022274F5202274E1A60274B1D5D50
:109F6000002D21D0A31E012B03D80121E0B2FFF761
:109F70001DFF012D18D11F4B9B69E3402B4213D0CD
:109F8000E3B218000193FFF711FE01000198FFF7FB
:109F90004DFFE3B2143B022B1DD801217156184A24
:109FA0008D405369AB4353613B7F002B0DD0E5B22D
:109FB0002800FFF793FF2800FFF7F8FD7B7F0100E3
:109FC000834202D02800FFF78FFD01340C370236A0
:109FD000172CC3D1F7BD012100237156F3568D40D4
:109FE000074A9B009B189A68AA439A60DCE7C04620
:109FF00000E100E07067FF1F51B900117167FF1F9A
:10A0000000F0004010B504000520162C0CD80121EA
:10A010002000FFF7DBFE0123044A002011194B70DA
:10A02000A34091690B43936110BDC0467067FF1F49
:10A0300070B50E0015000400FFF70EFF0C236343FC
:10A04000094A20009B189D605E60FFF747FFF021E2
:10A05000064B074A8900051E5A5002D02000FFF720
:10A06000FBFE280070BDC0468C67FF1F0000FF1F6D
:10A07000499B001170B5134D07202C78002C1FD17F
:10A08000982221005200280001F03EFA0123C4204A
:10A09000FF222B700C4B80001C635C630B4B1C601D
:10A0A0005C600B4B195891437F3A0A431A50802247
:10A0B00052021A600D20074A074901F02DF92000CD
:10A0C00070BDC0467067FF1F00800040A0F00040D8
:10A0D00000E100E03D9F0011299D0011030010B533
:10A0E0000620072B09D8054A137000F0EDFFD72191
:10A0F0000020034B034A89005A5010BDB044FF1F93
:10A100000000FF1F151BFF1F70B51D0002240C2946
:10A1100010D8094ACA40D2070CD5FBF725FF041E08
:10A1200008D1059A04992800FBF73AFFFCF7A8FD2F
:10A13000FFF7F8FA200070BD1210000030B50D785E
:10A1400002232C009C43184201D02B431C000825FD
:10A150002300AB43284201D02B00234320241D00C1
:10A16000A543204201D01C4325002A230D7018422C
:10A1700004D011781E3B0B43137030BD0028FCD176
:10A180000C2113788B43F7E7F8B51D0006AB1B884D
:10A19000140007AA0E000B201778002B27D10A788D
:10A1A000022A49D14A68507811780002244A0843AB
:10A1B0008018042840D801F067F803121D1B230003
:10A1C000F06801F0B1F8021CC0B2B84200D93A1CE4
:10A1D000D2B22000F1682A8001F02EFA06E00222B5
:10A1E000F3681B882A8023701B0A63700020F8BD67
:10A1F0000622EEE701232B80F3681B782370F5E736
:10A20000F368002B16D008222A801A8822701A8838
:10A21000120A62705A88A2705A88120AE2709A88EA
:10A2200022719A88120A6271DA88A271DB881B0A8D
:10A23000E371DBE72B80D9E701202B80D7E7C0460D
:10A2400000D6FFFFF7B516000A781D0008AB1F887F
:10A250000C000123022A18D14A68507811780002B4
:10A260002B4A0843801803280FD801F00DF8022567
:10A270004439E06801F058F8C0B20723B84204D36B
:10A280007B190193152B02DD0D231800FEBDE0683C
:10A290002A003100C01901F0CFF96B4600209B88DD
:10A2A000E268D0541B4B1B68834203D01B68834277
:10A2B00000D098470023E8E70B23002FE5D1022DBB
:10A2C000E2D1737832781B021343E2681380114B9A
:10A2D0001B68002BEED01B68002BEBD00120E8E7B9
:10A2E0000B23002FD1D1062DCED12A003100E068FA
:10A2F00001F0A2F9DEE70B23002FC6D1012DC3D157
:10A3000032787533012AC0D8E3681A70D2E7C046A4
:10A3100000D6FFFF7C69FF1F70B50C0015000728F1
:10A3200037D800F0B1FF041436361B36242E18201F
:10A3300015290BD8184E16220021300001F044F9DF
:10A3400022002900300001F077F9002070BD1820AC
:10A350000229FBD11288114B1A80F6E71820082930
:10A36000F4D10A000E48290000F0E6FEEDE71820BF
:10A370000129EBD10B4B10780B49DA69FFF7DEFEB0
:10A38000E3E718200129E1D1064B10780749DA6B81
:10A39000F4E70220DAE7C0466469FF1F2E45FF1F7D
:10A3A0002445FF1FB444FF1FDC44FF1FFC44FF1F74
:10A3B000030010B50020DB0704D50721024A03483B
:10A3C00000F08CF810BDC046DCB90011B444FF1F8A
:10A3D000054A03001068002803D082889A4201D100
:10A3E000806870470068F6E7806BFF1F0A880300EB
:10A3F00008009A4204D08A8804309A4200D0002093
:10A4000070470000F8B5F82200230D4F0D4E796813
:10A41000050042433370994200D07B600A4C002112
:10A42000200001F0D1F800231A007C60AB4202D179
:10A4300000203370F8BD01332280DBB2F834F5E739
:10A44000806CFF1F7C6CFF1F846BFF1F73B56B4616
:10A4500001900600684615001980FCF743FF041EB2
:10A4600011D1002D0FD07689002E11D00C2000F0D4
:10A470004BFF00280ED0084A046013688680856070
:10A48000002B02D11060200076BD1A001B68F7E790
:10A490000224F8E71324F6E7806BFF1F0121002256
:10A4A0000A4B10B549420A4C198099809A719A70EA
:10A4B000084B2070012019805A60FFF7A3FF207815
:10A4C000FCF76EFF0448FDF719FF10BD8469FF1FFC
:10A4D000886CFF1F806CFF1F89A50011022310B537
:10A4E000002802D0FFF7B2FF0300180010BD0000E3
:10A4F000030010B50020DB0704D50421024A0348FD
:10A50000FFF7A4FF10BDC046F0B900113445FF1F8E
:10A51000F0B50E2687B003930CAB1F8802ABF6187C
:10A520000500080031000292FDF75EF804000120EA
:10A53000002C0FD03088FFF74BFF03000E20002BBC
:10A5400008D05E68002E05D021002800039B029AE7
:10A550000097B04707B0F0BD0A4B10B5984207D13D
:10A560000122002352420A808B708A808B7110BDB9
:10A57000FFF73CFF0028FAD001235B420380002351
:10A580008370F4E7FFFF0000F8B5050001290AD148
:10A59000134E00243388F827AB4219D02800114904
:10A5A000FFF7DAFF06E0022904D10139FDF724FFA5
:10A5B0000028EDD0F8BD3B0063437268D018D35A31
:10A5C000002B09D03A00002100F0FEFF0134E4B274
:10A5D000054B1B78A342EED801235B423380DDE7B5
:10A5E000806CFF1F8469FF1F7C6CFF1F10B5FFF795
:10A5F000FDFE03000020834200D0987810BD0000CB
:10A60000F0B589B01C000EAB80CB03901E8810AB58
:10A610001B78049202930B7A0D00DB0616D42B787C
:10A620000593022B24D00498FFF7D2FE002812D005
:10A6300003689C46002B0ED0029B22000193290048
:10A640003B00644603980096A04705E00498FFF796
:10A65000BFFE002802D10E2009B0F0BD8368002B98
:10A66000F9D00A222900039898470028D7D0F3E7A9
:10A670006B6858781A786B4B000210439842D2D816
:10A68000043B984210D2684B984242D015D8674B91
:10A69000C0180128C7D80B20002EDDD1EB681A782E
:10A6A00059683A80200028E0614BC018032800D97F
:10A6B00079E000F0E9FD846A789E5E4B9842B2D161
:10A6C0000B20002EC8D101233B80EB6831001B78A2
:10A6D00023706889013080B2FCF786FF3A88031E38
:10A6E0000ED0017802328A183A804289627042891B
:10A6F000120AA27059680278E01C00F09DFF06E083
:10A7000004323A8031000422601C00F05DFF00201A
:10A71000A2E70B20002E9FD1EB6807A91E88042317
:10A720003B80330A300026706370FCF75DFF051E26
:10A7300028D004AB9A890E2304A95B183E49C66849
:10A74000FCF7C6FF00280BD12B783C486A680599B6
:10A75000FBF77CFB002803D1012304AA5B42D381D1
:10A760003278022A06D17168201D00F065FF3B880F
:10A7700002333B800E2304AA9B181B88A3701B0A7C
:10A78000E370C4E704ABDE81F4E70B20002E00D0B9
:10A7900062E7E9680398FFF729FF02233B802070F6
:10A7A000000A6070B3E70B20002E00D054E70222AD
:10A7B000EB681B883A8023701B0A6370A7E7E86880
:10A7C00000F0B2FDC2B203000720B24200D243E75C
:10A7D0000DD00299DBB27118994202DB921BD3B201
:10A7E0000293029BE9681A003B8089195AE700230B
:10A7F000F6E70B20002E00D02EE70722EB683A8008
:10A800001A7822705A7862705A88A2705A88120A8E
:10A81000E2701A792271DA886271DB881B0AA371EF
:10A8200075E7C046042900000228000000D8FFFF99
:10A83000FFD6FFFF03280000FFFF000020B9001132
:10A84000F0B58DB06B460020089120229B5E8342BC
:10A850003DDAA64B187800F047FE071E32D0037889
:10A86000B02B2CD10079023816281FD800F09CFE9E
:10A8700017001E001E001E0031001E0096001E0064
:10A880001D011E0052011E0073011E00CD011E009D
:10A8900050021E001E001E008E021E00E302944B9A
:10A8A00094491B8878880B80FBF710F83800FCF778
:10A8B00081FF914B1B68002B01D03800984738006E
:10A8C00000F012FC8020089B0002434018000DB0ED
:10A8D000F0BDF6220021874800F076FE0BAA3B7BF4
:10A8E0007989388900923A000D32FCF795FD040011
:10A8F000804B1B78002C3FD146E0804B7888059335
:10A900007F4B4100CB5A0BAE073BDBB23288029340
:10A91000002301937B4B210006930093059BFFF7D7
:10A920006FFE744D002810D1069B3A8A1B889A420C
:10A930000BD138000599123000F056FD002804D0E4
:10A940002B7862899B00EB185A80162306A81B18E7
:10A95000328820007989FCF7BBFE2B7804009A002E
:10A96000AA1851880029C3D00133DBB22B7000280C
:10A9700007D006A9C98A9180634A12889A42BCD836
:10A9800002E0012149429180002B04D05949788886
:10A99000FAF7D0FF8AE73E890A2479E000253E894C
:10A9A000574B06937B88069A5B009B5A033B9D425C
:10A9B00002DB002DF0D05BE0162206A812183B7BCC
:10A9C000798900923A0030000D32FCF725FD0590A0
:10A9D000002858D04689017A7888FCF7E7FC041EE5
:10A9E00044D1464B78880793069B4100C95A454B92
:10A9F0000439C9B206AAD28A06930291019400933F
:10AA00000599079BFFF7FCFD041E2FD1069B3949D2
:10AA10001A88931C002D26D14B807988384B490029
:10AA2000CB5A5119033B8B4220DD059B31485B8992
:10AA300041190B71A91C0135C9B2EDB20591451937
:10AA40001B0A2B71059B2D490433181800F0F4FDE7
:10AA50002C4B059A1B88D318DDB22C4B9E4205D097
:10AA60000136B6B29CE749889942D6D0002D0CD069
:10AA7000204C2800618800F05FFC2070210078885D
:10AA8000FAF768FF12E7059CF0E7002C00D183E796
:10AA90007B78142B00D109E716493B794E800B7067
:10AAA0000C717888FAF708FF00E7162406ABE41863
:10AAB00021003889FCF798FD011E00D1B7E17888A4
:10AAC00022880F4C45002C5B0A4D013CE4B20294F5
:10AAD00000240F4B01940095FFF792FD041E00D057
:10AAE00014E129007888FAF745FFDFE6886CFF1F3C
:10AAF0002044FF1F8C69FF1F8069FF1F866AFF1FAC
:10AB0000BC65FF1F7C6BFF1F1E44FF1FFFFF000083
:10AB10008E69FF1F162406ABE41821003889FCF764
:10AB200063FD011E00D182E178882288AE4C450089
:10AB30002C5BAE4D013CE4B202947C89AC4B019499
:10AB40000095FFF75DFD041E00D0DFE02900788846
:10AB5000FAF71AFFAAE60025A44B1D803B00FE333E
:10AB60001B78A24A78880792AB4208D99E4B12887C
:10AB70000693069943005B5A013B9A4203DB07990F
:10AB8000FAF70CFF92E616246B00FB18059306AB50
:10AB9000E418059B21001889FCF726FD011E03D14E
:10ABA000059B01241E8973E77888924B2288069CB6
:10ABB000099343001B5B904E013BDBB202930023E1
:10ABC00000960193099BFFF71BFD041E02D0059B15
:10ABD0001E895DE77B88069A5B009B5A079A10885E
:10ABE00032881218934202DC1B1A013B33807F4CDF
:10ABF000023032880999001900F01EFD238832883E
:10AC000001359B182380EDB2A8E70BAA3B7B79891D
:10AC1000388900923A000D32FCF7FEFB00250590C2
:10AC2000059B002B04D10A24002D00D16EE060E0CA
:10AC3000059B7888197AFCF7B9FB0100041E63D1E3
:10AC4000694C6C4B788806940993069B4400E45A3F
:10AC5000694B063CE4B20BAE328807930294019133
:10AC600000930599099BFFF7CBFC041E4CD1079B71
:10AC70005E491B881A1D002D30D14A80059B5B4C14
:10AC80005A8963191A716B1C9BB2E318120A1A7164
:10AC9000162306A832881B1879890598FCF718FD39
:10ACA000FF21AA1C2E1D03350B00059092B2B6B2EF
:10ACB000ADB2002803D006ABDB8AD9B21B0AA218BA
:10ACC000651911712B714C4D301D2A884949201886
:10ACD00000F0B2FC2B88F618B5B2A1E74988914282
:10ACE00007D17A8806995200525AEB18053A9A42CF
:10ACF000C4DC3E4C2800618800F09EFA20702100E0
:10AD00007888FAF755FED1E5002DF2D13E89BFE6ED
:10AD1000162606ABF61831003889FCF765FC3D00B5
:10AD20000400FF3500282DD0037A9B060CD40022A6
:10AD30007B893989788800923A000C32FFF7E8FB6A
:10AD4000041E10D03E8915E03088FFF741FB002833
:10AD50001AD08368002B17D02100122278889847D8
:10AD6000041EE4D0EEE7AB78002B02D17888FAF726
:10AD70002FFE0026AB78002B00D097E5002C00D1E9
:10AD800094E585E60124DDE70E24DBE7162506AB16
:10AD9000ED1829003889FCF727FC041E47D0037AF8
:10ADA0009B0611D4154A7B881188994203D0144818
:10ADB000814207D11380134BF8261D780023D9B2A6
:10ADC000A94221D30924A1E72888FFF701FB002825
:10ADD0002FD08368002B2CD021001222788898472E
:10ADE000041EDFD092E7C046BC65FF1F8C69FF1FC1
:10ADF0008E69FF1F866AFF1F7C6BFF1F806CFF1F21
:10AE0000FFFF00007C6CFF1F310059435468013381
:10AE10006018615A0029D2D13C0008342100F82280
:10AE200000F00AFC21007888FAF7DAFD3EE50124FB
:10AE30006CE70E246AE71D4B1A887B889A4231D052
:10AE40007888FAF7D7FD31E5F82305985168434330
:10AE5000CD18C95A00291FD03B7A012B0BD16C8821
:10AE6000AB887888AA1D0094FFF752FB041E02D01D
:10AE700000233B722E88F8220021280000F0A4FB5A
:10AE800000232B80059B0133DBB20593084B05990A
:10AE90001B78064A8B42D7D801235B421380002CD3
:10AEA000CED0F5E5002634000596EFE7806CFF1F55
:10AEB0007C6CFF1F70B504000E001500FFF796FABA
:10AEC000031E08D131000548FFF790FA0300112056
:10AED000002B02D01C8000209D7070BDFFFF000081
:10AEE000F8B50B4F06003B780D001400FF2B0ED079
:10AEF0000A2000F079F9011E09D0B1230380002354
:10AF000046800371C5800481387800F0FDF8F8BDF3
:10AF10007545FF1FF7B50F0008A90600088809A9A5
:10AF20000B240988002821D10234022B1ED1557828
:10AF300013782D021D432B008B4301937334002B98
:10AF400014D1FB68300019000093FFF74FFB019C00
:10AF500085420BD02A0030000099FFF7ABFF041E9A
:10AF600004D12A0030007989FFF7BAFF2000FEBD26
:10AF7000F0B50E7885B003900AA805880120022E4E
:10AF80000DD14C682778647824023C43054FBC42BD
:10AF900005D10398DBB201960095FFF7BBFF05B022
:10AFA000F0BDC0460229000010B504000C4800F0B6
:10AFB0008BFA0C48A16B00F087FA0B48E16B00F0AC
:10AFC00083FA0A48216C00F07FFA094B0948196896
:10AFD00000F07AFA084B1B68002B00D09847FEE778
:10AFE000F2B7001108B8001117B8001126B8001107
:10AFF00004ED00E035B800118C6CFF1F002307B58D
:10B0000001A80193FFF7D0FF044A0548002110B5BD
:10B01000121A00F0D9FAF8F7CBFCFEE7906CFF1F8C
:10B020007845FF1F0000000001B40248844601BCBF
:10B03000604700BF017F000001B40248844601BCA4
:10B04000604700BF6939FF1F01B40248844601BC54
:10B05000604700BFB14E000001B40248844601BC05
:10B06000604700BFC926000001B40248844601BC05
:10B07000604700BF8D12000001B40248844601BC45
:10B08000604700BF213AFF1F01B40248844601BC5B
:10B09000604700BF8552010001B40248844601BCEC
:10B0A000604700BF691F000001B40248844601BC2C
:10B0B000604700BF6932FF1F01B40248844601BCEB
:10B0C000604700BF456B010001B40248844601BCE3
:10B0D000604700BF151BFF1F01B40248844601BC36
:10B0E000604700BFC9A9000001B40248844601BC02
:10B0F000604700BF434D010001B40248844601BCD3
:10B10000604700BFA946010001B40248844601BC63
:10B11000604700BF594F010001B40248844601BC9A
:10B12000604700BF093BFF1F01B40248844601BCD1
:10B13000604700BF9130FF1F01B40248844601BC44
:10B14000604700BF810E000001B40248844601BC84
:10B15000604700BF5539FF1F01B40248844601BC57
:10B16000604700BFA139FF1F01B40248844601BCFB
:10B17000604700BFF30E000001B40248844601BCE2
:10B18000604700BF2526000001B40248844601BC88
:10B19000604700BF291C000001B40248844601BC7E
:10B1A000604700BF3D18000001B40248844601BC5E
:10B1B000604700BF313CFF1F01B40248844601BC18
:10B1C000604700BF4134FF1F01B40248844601BC00
:10B1D000604700BF851F000001B40248844601BCDF
:10B1E000604700BFE548000001B40248844601BC46
:10B1F000604700BF1D4D010001B40248844601BCF8
:10B20000604700BFC521000001B40248844601BC6C
:10B21000604700BFED4A010001B40248844601BC0A
:10B22000604700BFA134FF1F01B40248844601BC3F
:10B23000604700BFC132FF1F01B40248844601BC11
:10B24000604700BF090E000001B40248844601BCFB
:10B25000604700BF8132FF1F01B40248844601BC31
:10B26000604700BFA54F010001B40248844601BCFD
:10B27000604700BF090E000001B40248844601BCCB
:10B28000604700BF2951010001B40248844601BC57
:10B29000604700BF453CFF1F01B40248844601BC23
:10B2A000604700BF056A000001B40248844601BC43
:10B2B000604700BFE117000001B40248844601BCAA
:10B2C000604700BF4D1F000001B40248844601BC26
:10B2D000604700BF2146010001B40248844601BC1A
:10B2E000604700BF2124000001B40248844601BC2D
:10B2F000604700BFEDA5000001B40248844601BCD0
:10B30000604700BF311B000001B40248844601BC05
:10B31000604700BF3D4B010001B40248844601BCB8
:10B32000604700BF0933FF1F01B40248844601BCD7
:10B33000604700BFDD52010001B40248844601BCF1
:10B34000604700BF350E000001B40248844601BCCE
:10B35000604700BF5549010001B40248844601BC62
:10B36000604700BF9DA9000001B40248844601BCAB
:10B37000604700BF3555000001B40248844601BC57
:10B38000604700BF0134FF1F01B40248844601BC7E
:10B39000604700BF0189000001B40248844601BC37
:10B3A000604700BFC94A010001B40248844601BC9D
:10B3B000604700BF5D17000001B40248844601BC2D
:10B3C000604700BF0124000001B40248844601BC6C
:10B3D000604700BF1D4B010001B40248844601BC18
:10B3E000604700BF7918000001B40248844601BCE0
:10B3F000604700BFCD4C010001B40248844601BC47
:10B40000604700BFC53F000001B40248844601BC4C
:10B41000604700BF1537FF1F01B40248844601BCD6
:10B42000604700BFF136FF1F01B40248844601BCEB
:10B43000604700BF5952010001B40248844601BC74
:10B44000604700BF0D52010001B40248844601BCB0
:10B45000604700BF8B52010001B40248844601BC22
:10B46000604700BF7D18FF1F01B40248844601BC3D
:10B47000604700BFD1A5000001B40248844601BC6A
:10B48000604700BFC95C010001B40248844601BCAA
:10B49000604700BF055E000001B40248844601BC5D
:10B4A000604700BF75A9000001B40248844601BC92
:10B4B000604700BF9938FF1F01B40248844601BCB1
:10B4C000604700BFB352010001B40248844601BC8A
:10B4D000604700BFE53A010001B40248844601BC60
:10B4E000604700BFE537FF1F01B40248844601BC36
:10B4F000604700BFF54E010001B40248844601BC1C
:10B50000604700BF091B000001B40248844601BC2B
:10B51000604700BFB70E000001B40248844601BC7A
:10B52000604700BFC56D010001B40248844601BCFC
:10B53000604700BF6DBC000001B40248844601BCF6
:10B54000604700BFADAE000001B40248844601BCB4
:10B55000604700BF1147010001B40248844601BCA6
:10B56000604700BF4551010001B40248844601BC58
:10B57000604700BF5118FF1F01B40248844601BC58
:10B58000604700BF014C010001B40248844601BC81
:10B59000604700BF9135FF1F01B40248844601BCDB
:10B5A000604700BFDD30FF1F01B40248844601BC84
:10B5B000604700BF593CFF1F01B40248844601BCEC
:10B5C000604700BF5147010001B40248844601BCF6
:10B5D000604700BF154D010001B40248844601BC1C
:10B5E000604700BF5522000001B40248844601BCF8
:10B5F000604700BFD949010001B40248844601BC3C
:10B60000604700BFD91B000001B40248844601BC5A
:10B61000604700BFE139FF1F01B40248844601BC06
:10B62000604700BFE928000001B40248844601BC1D
:10B63000604700BF5125000001B40248844601BCA8
:10B64000604700BFE94C010001B40248844601BCD8
:10B65000604700BF4550000001B40248844601BC69
:10B66000604700BF353BFF1F01B40248844601BC60
:10B67000604700BFB54C010001B40248844601BCDC
:10B68000604700BFF94C010001B40248844601BC88
:10B69000604700BF8D3AFF1F01B40248844601BCD9
:10B6A000604700BF6571010001B40248844601BCD7
:08B6B000604700BFC51D00004A
:10B6B8000002010302030303040305020602070252
:10B6C800080209000A030B030C020D020E030F0304
:10B6D800100311031303140315001600793D00111C
:10B6E800AD3D00110000000002000000FAB6001194
:10B6F800192A0F180A000000F1590000FD24000063
:10B7080041460100057A0011199A00118D6E001149
:10B71800097800112150001141A80011DD4C0011D9
:10B72800713F0011A1400011000000001616000032
:10B738000200000044B70011F4FFF3FFD2FC000040
:10B748005D4100110000000000000000547579619F
:10B758000056302E37003030303100676974687514
:10B76800622E636F6D2F70767678004254483031C0
:10B77800000000000200000090B70011292A282AC2
:10B78800272A262A252A242A0A180000E20400006B
:10B798007102000078EC00007440000010270000DF
:10B7A80060F0000006640000204E00000000000069
:10B7B800000000001F501D000206B4000001140024
:10B7C8000700000083020000303132333435363749
:10B7D8003839414243444546005048592B3632587F
:10B7E80058504C555330353034005B4861726420F2
:10B7F8006661756C742068616E646C65725D0A00C0
:10B808004C522020203D203078253038780A0050CE
:10B81800432020203D203078253038780A005053C6
:10B828005220203D203078253038780A004943538B
:10B8380052203D203078253038780A0031540011E4
:10B848008554001100000000020000005CB80011DF
:10B858006F2A6E2A1A18000001A0000000000000DC
:10B868006410B71DC8206E3BAC30D9269041DC76F9
:10B87800F4516B6B5861B24D3C7105502083B8EDA3
:10B8880044930FF0E8A3D6D68CB361CBB0C2649BC7
:10B89800D4D2D38678E20AA01CF2BDBDFB349B5FEC
:10B8A8008000008000100000000000008F5A001186
:10B8B80019710011B35A001121750011375B00117D
:10B8C800F7740011AD5B0011CD740011FF5B00111E
:10B8D80095760011675C001195760011995C00114E
:10B8E8004F760011AD5B001185740011255C0011C5
:10B8F8002D76001100000000000000000B5D001113
:10B908002D7600116D5D001131710011052A042A90
:10B91800012A002A022903280128002801180018F2
:10B928000000000000000000000000000000008788
:10B9380001010201020101020102030304010301E2
:10B94800010101010303020103000D000E001000B4
:10B95800110013001401070108010A010B011C0161
:10B968001D02040205020702080219021A021C023B
:10B978001D03010302031700020100050400080764
:10B98800000B0A001716001D1C0102010105040125
:10B998000E0D011110011413011716011A190202D4
:10B9A80001020B0A020E0D021110021413021716DF
:10B9B800030504030807030B0A030E0D0001020325
:10B9C80007090A0B0E0F101112141718191A1B1F4A
:10B9D8002021220089A1001145A2001100000000C9
:10B9E8000200000026B900110000000071AF00112C
:0CB9F800000000000200000024B9001153
:020000041FFFDC
:1000000000000000D53E001100B70011FCB6001141
:100010008462FF1F000000000000000000000000DC
:1000200000000000000000000000000000000000D0
:1000300000000000000000000000000000000000C0
:1000400000000000000000000000000000000000B0
:1000500000000000000000000000000000000000A0
:100060000000000000000000000000000000000090
:100070000000000000000000000000000000000080
:100080000000000000000000000000000000000070
:100090000000000000000000000000000000000060
:1000A0000000000000000000000000000000000050
:1000B0000000000000000000000000000000000040
:1000C0000000000000000000000000000000000030
:1000D0000000000000000000000000000000000020
:1000E0000000000000000000000000000000000010
:1000F0000000000000000000000000000000000000
:1001000000000000000000000000000000000000EF
:1001100000000000000000000000000000000000DF
:1001200000000000000000000000000000000000CF
:1001300000000000000000000000000000000000BF
:1001400000000000000000000000000000000000AF
:10015000000000000000000000000000000000009F
:10016000000000000000000000000000000000008F
:10017000000000000000000000000000000000007F
:10018000000000000000000000000000000000006F
:100190006534FF1F5533FF1FC166010000000000DA
:1001A000000000000000000000000000000000004F
:1001B000000000000000000000000000000000003F
:1001C000000000000000000000000000000000002F
:1001D000000000000000000000000000000000001F
:1001E000000000000000000000000000000000000F
:1001F00000000000000000000000000000000000FF
:1002000000000000000000000000000000000000EE
:1002100000000000000000000000000000000000DE
:1002200000000000000000000000000000000000CE
:1002300000000000000000000000000000000000BE
:1002400000000000000000000000000000000000AE
:10025000000000000000000000000000000000009E
:10026000000000000000000000000000000000008E
:10027000000000000000000000000000000000007E
:10028000000000000000000000000000000000006E
:10029000000000000000000000000000000000005E
:1002A000000000000000000000000000000000004E
:1002B000000000000000000000000000000000003E
:1002C000000000000000000000000000000000002E
:1002D000000000000000000000000000000000001E
:1002E000000000000000000000000000000000000E
:1002F00000000000000000000000000000000000FE
:1003000000000000000000000000000000000000ED
:1003100000000000000000000000000000000000DD
:1003200000000000000000000000000000000000CD
:1003300000000000000000000000000000000000BD
:1003400000000000000000000000000000000000AD
:10035000000000000000000000000000000000009D
:10036000000000000000000000000000000000008D
:10037000FDAF0011000000000000000000000000C0
:10038000000000000000000000000000000000006D
:10039000000000000000000000000000000000005D
:1003A000000000000000000000000000951AFF1F80
:1003B000000000000000000000000000000000003D
:1003C000000000000000000000000000000000002D
:1003D000000000000000000000000000000000001D
:1003E000000000000000000000000000000000000D
:1003F00000000000000000000000000000000000FD
:081838009070FF1F4118FF1F13
:10184000024981F3088802F04BFA00009070FF1FF4
:1018500010B502F00DFA072804D0122808D002288B
:1018600008D010BD044A0420136B01331363F8E75A
:101870000220F6E71420F4E76466FF1FF8B50700BE
:101880000C0026002500503630785135002804D150
:101890000300287058342370F8BD2978CA00481E08
:1018A0008141A3183800A25C5B68C9B2FFF7D0FF82
:1018B00000280DD12B78DA00A218013350602B706C
:1018C0003378044A013B3370136A01331362D8E75B
:1018D0000123DFE76466FF1F5C234343074910B51C
:1018E000C9180B0058331B78012B05D1FFF7C6FF31
:1018F000034A936A0133936210BDC0469866FF1F86
:101900006466FF1F10B502F0C3FA064A01211300F6
:1019100010CB4942D967044B136002F009FB200049
:1019200010BDC04600E100E01000100010B504003A
:1019300002F0AEFA024B1C6002F0FAFA10BDC0468B
:1019400000E100E010B5040002F0A2FA4021094ACB
:10195000200013688B43136002F062FB01F064FD0A
:101960000022054B01201A60044B04321A6002F079
:1019700097FAFEE71CF00040C4F00040C0F00040C1
:10198000431E5A425341A022F0B5D2015B4213409C
:10199000154D164A40019B182A18127E8BB00191F2
:1019A000002A1BD01A000832D46F0022E6B206AF1C
:1019B000E4B294420EDC2818C369002B08D00199C8
:1019C00002AA117106AA049202AA167303A89847E4
:1019D0000BB0F0BD1978B9540132EAE71A7D1A78D4
:1019E00006AB01261A70E6E72469FF1F004000409D
:1019F000F0B5254B04004001C25C85B0002A2BD015
:101A00001A18117E002927D0917E002924D011793F
:101A1000022921D11689D788D168F51BADB22A1CBD
:101A2000102D00D9102292B2BE4217D118180123EE
:101A300003710023C269C38003819A4206D06846BD
:101A4000032103730171029301A890470820002C21
:101A500000D0192001F034FC05B0F0BD013C654216
:101A60006C41A0256442ED012C40084D1B186419FF
:101A7000074D0633013A92B2AA42EDD01888461CAF
:101A80001E80085C2070F5E72469FF1F00400040BD
:101A9000FFFF00000F220E4B10B59868104002386F
:101AA0000A280BD802F0CEF80D0A0B0A0A110A0A0E
:101AB0000A0A060002210020FFF762FF10BD012183
:101AC000F9E70020FFF794FFF8E7DB6FF6E7C04681
:101AD000004000400F220E4B10B5986810400238AD
:101AE0000A280BD802F0AEF80E0A0B0A0A120A0AEC
:101AF0000A0A060002210120FFF742FF10BD012162
:101B00000800F9E70120FFF773FFF7E7DB6FF5E760
:101B10000090004013B5334C2378072B3DD8324B4F
:101B20001A78324B002A39D18022196852020A43AE
:101B30001A60252001F034FF20232D4A11680B4341
:101B4000802113606B460422C905086807331042E0
:101B500028D080210422C905C86810422ED08021D7
:101B60002020C905CA688243CA6014221A701A78F4
:101B7000002A2FD18021C905C86820320243CA60DB
:101B800014221A701A78002A28D11A4B1A7D22784A
:101B90005A601D221A705932DA6013BD1A6816494C
:101BA0000A40C5E7086802430A6014221A701A78CE
:101BB000002ACED01A78013AD2B2F7E7C8680243B9
:101BC000CA6014221A7019784A1ED2B21A700029FB
:101BD000F9D1C4E71A78013AD2B2C7E71A78013AC4
:101BE000D2B2CEE7B044FF1F7845FF1F3CF0004063
:101BF000A844FF1F00200040FFFFFEFF564B70B5BA
:101C00001B68012B03D1554A936D0133936502F094
:101C1000CFFA534B534A1860534B544C1A6001236C
:101C2000534A1360534A13602378002B06D00622D0
:101C30005149524802F0ACF900232370504A514BED
:101C400010681B78C1B2002B0ED14F4CC0B2237864
:101C50005BB2002B4FDB237824785BB264B21B04A9
:101C600024021B191B1813600B1C50294ED950233A
:101C7000464A47491078DBB2FF2202284BD1086858
:101C8000444C454D267890432A78964254D9227880
:101C900024782E78023B5D10A31B6B435201D31AAC
:101CA00010335B111843086002F052F8031F012B38
:101CB00045D83A4B1B78002B06D0394B1B78002BAC
:101CC00002D0002002F04CF9A122364B9200997804
:101CD000354B4A431B689B18832292009B181B7844
:101CE000033B012B03D8AF20400002F011F8012282
:101CF0002E4BDA8270BD237824785BB264B2FF3356
:101D0000FF341B0424021B190138ABE7CAB2022AB4
:101D1000AED20223ACE70868254C264D26789043C6
:101D20002A78964208D9227824782D78023B5B10D5
:101D3000641B63435201B2E72378DBB2B2E70228A7
:101D4000D5D11D4B1B78013B022B03D91B4B1B78B4
:101D5000022BCCD16C20C8E79809FF1FFC0FFF1F96
:101D60009C65FF1FFF3F000014100340A065FF1F8C
:101D70000C10034000100340D50BFF1F7211FF1F12
:101D8000B40003408C09FF1F680AFF1F490AFF1FA8
:101D900094000340460AFF1F470AFF1FF908FF1F70
:101DA0002209FF1F300DFF1F3409FF1FBC0BFF1F4F
:101DB000440AFF1F450AFF1F1C09FF1F2309FF1FBD
:101DC00010B502F025F90022014B1A8010BDC04663
:101DD0009865FF1F10B502F093F8A121054A89000C
:101DE0009478054A61431268044B5218528C1A8049
:101DF00010BDC046300DFF1F3409FF1F9865FF1F3F
:101E000010B50D4B0D4A9978A1239B004B431268E6
:101E1000D218531DD97F0A4B1B88994209D2441C02
:101E200007D0C82805D0D2695B1A5A43054B5343E3
:101E3000C01801F0A5FF10BD300DFF1F3409FF1FB2
:101E40009865FF1F7102000070B5244D2B68002BB0
:101E500028D001F06DFF2B68D8402B680400002BC0
:101E600027D001F0FDFF2B68D8401D4B1D4A997803
:101E7000A1239B004B431268D118D25C91239B0095
:101E8000002A20D0CA580132CA50174B17491B6884
:101E90000868834214D3D23B181A012A1AD0144B73
:101EA000186070BD01F044FF124B196802F080F811
:101EB000D3E701F0D5FF0F4B196802F079F8D4E7AA
:101EC0000D495B18E8E7CA500C4B1B68DB68E41847
:101ED000201AE4E7F530FF30E1E7C0461C08FF1F99
:101EE000300DFF1F3409FF1F9C09FF1F9C65FF1F5A
:101EF000A009FF1F1808FF1F2DFF3F00A465FF1F4B
:101F000070B504000D00282916D10300A433C2883F
:101F10001B889B1A0B4A9BB293420DD906006A3666
:101F200005223100653001F00BFF002804D131009B
:101F3000200001F0CDFE70BD2900200002F028F93C
:101F4000F9E7C046FE7F0000F8B50400012002F06A
:101F500047F801F04DFF174A174910600968030060
:101F60001648174E01601748776805680020AF4291
:101F700001D27068281A144D091928601348C162EB
:101F8000A421446A49032143416211490978002987
:101F900005D010490978022902D10F3B1360F8BD22
:101FA000012901D1083BF9E7032901D1053BF5E7F8
:101FB000033BF3E7E408FF1F28F00040340AFF1F4B
:101FC00028100040180AFF1F1C0AFF1F00F00040E5
:101FD0001C09FF1F4A0AFF1F70B580241025E40565
:101FE000A3682B43A36002F0B3F8A368AB43A360DC
:101FF00070BD0000F7B5160080221C001023D2052A
:102000000191916805000B43936000225A4BD73031
:102010001A6002F04DF89D232A002F009B00EB5818
:10202000CA3201210092FC37002B01D00021009A16
:10203000386801F03DFE2900009BCB311A784F4BE8
:10204000D3351A604B780A781B0213438A7812043E
:102050001A43CB781B061343494A1BBA13604B79CA
:102060000A791B0213438A7912041A43CB7931008F
:102070001B061343434A1BBA13606B782A781B0272
:102080001343AA7812041A43EB781B0613433E4A03
:102090001BBA1360019A330213433C4A13603C4B52
:1020A00022001B1B9C4603293DDCB3089A00130049
:1020B0005142B21A032A46D1354AE018511A8278A1
:1020C0004078120400020243E05C043302430A60D9
:1020D0000022FF2B4BDDF0222E4B12011A600F2243
:1020E0002D4B1A602D4A1368002BFCD00023224A86
:1020F00027491360091B321D0B191B68043A180A83
:1021000023706070180C1B0EA070E3700434002A5A
:10211000F2DC802210213B68D20501333B609368DA
:102120008B439360F7BD6346D578981893782D0656
:102130001B042B43157804392B43557804322D02A8
:102140002B430360AFE7022A0AD1114AE05C511A1F
:10215000E2185278120202430A6004339BB2B7E7D6
:10216000012AB5D10A4A521AE15C1160F5E7084923
:1021700059180A600433ACE7000004403C000440F6
:102180003800044034000440300004400C00044097
:102190000001044004000440100004401400044006
:1021A000F7B5150080221C001023D205009191681C
:1021B00007000B4393600023654AD730136001F09A
:1021C00077FF9D233E009B00F9583B00CA36320042
:1021D000FC33002900D07FE0586801F069FD390028
:1021E00032785C4BCB311A604B780A781B02134370
:1021F0008A78AC4612041A43CB78281D1B06134379
:10220000554A1BBA13604B790A791B0213438A792A
:1022100012041A43CB791B061343504A1BBA1360AE
:102220004B7A0A7A1B0213438A7A12041A43CB7A36
:1022300021001B0613434A4A1BBA1360009A2B0263
:102240001343484A13602200474B1B1B0093009B1B
:10225000CE785B1801938B7836061B0433430E78D7
:10226000043833434E78043136023343019E3360E1
:102270000328ECDC0321A808431C9B0029408000B4
:1022800003292BD13849E5185E18A9786D78E35CED
:1022900009042D022943194331600300083300214A
:1022A000FF2B2DDD314B324919600F21314B196065
:1022B000012327490B60304B19680029FCD0062107
:1022C0001B680B40042B20D080220020D20593688D
:1022D0000A318B439360FEBD01217DE7022908D1BD
:1022E00021495D18E1184978E35C09021943296026
:1022F000D3E70129D3D11C495918E35C0B60CCE723
:102300001948181801600433CAE7002310490B600C
:102310006346002B0CDC3B00FC335A681021013271
:102320005A608022D205936801208B439360D2E7E4
:10233000009B9B181B68190A13705170190C1B0E17
:10234000D37004235B4291709C440432E0E7C046A2
:10235000000004403C0004403800044034000440C5
:10236000300004400C00044000010440040004401C
:10237000080F0000100004401400044070B5061E51
:1023800019D00222614B9B799343012B13D1604BEF
:102390001A78FF2A0FD15A78FF2A0CD19A78FF2A8F
:1023A00009D1DA78FF2A06D11A79FF2A03D15B799D
:1023B000FF2B00D1A7E0574B0C201A78012A08D038
:1023C0000022554D1A702B781A00093A042A01D8B8
:1023D000212070BD5A1F012AFAD94C4CA07B042839
:1023E00000D990E0A279032A00D98CE0821E012A4C
:1023F00003D862881F2A00D885E0002E61D0012E04
:1024000000D080E0A288012AE2D0002B0AD1013856
:10241000032803D801F016FC151D19151F202E7076
:1024200001F0D6FD2B785A1E032A16D800253B4B07
:102430001D602823237501F023FDA8422ED0A5801E
:10244000C6E7022320202B70EAE7042322202B700A
:10245000E6E7032321202B70E2E7073B012BB7D8E7
:102460002F4B1B68DB6A9B06B2D52E4B1A78002ACD
:10247000AED1A27B911E012901D9002AA8D1022246
:1024800080211A702823284D89012878237501F0AE
:102490006FFD80212878890101F0B2FC0123A3801F
:1024A000224B1B78002B0AD0FA228021204B92006D
:1024B0001B8809025A431C4B187801F0E9FD0020E3
:1024C00087E701F0E5FC2B78A680073B012B06D9B6
:1024D00018482E7001F03CFD1E2001F079FD114BD3
:1024E000114C1A78002A06D0802100222078890118
:1024F0001A7001F03DFD01F01BFD802120780902DA
:1025000001F036FDDBE7122063E7C046A60BFF1F94
:102510006B09FF1F1A09FF1F1C09FF1F4809FF1F36
:10252000A465FF1F2309FF1F1B09FF1F2109FF1FB0
:102530002C09FF1F0010004010B5002901D001F048
:102540004FFC10BDF7B5604B01919978A1239B001A
:102550004B435E4A060014681022E418D6235B0041
:10256000E0583623FF33E35C00279343222B41D10D
:10257000574B0F3A1A600760012501F009FC019BD7
:102580001880E8235B00E35C002B01D0B34258DDE8
:102590000023504FFB70AD33FF33E3581A68002A15
:1025A00003D09B88DB439B071DD03823FF33E35CBC
:1025B000002B18D09B235B00E35C002B13D1D1339D
:1025C000FF33E35CB3420EDAA4235B00E15AE01868
:1025D000090A023101F0F4FC23000122FE33013E1E
:1025E00001351A87FA70E8235B00E35C002B2AD0E0
:1025F000A8B2FEBD03683D00002BBED08188043028
:10260000090A023101F0DCFCD6235B00E3581F60AD
:10261000B2E72300B133BA00FF33985801378188FD
:102620000430090A023101F0CBFCE8235B00E35CD3
:10263000BB42EEDCE822F61AED1800235200A35448
:10264000A6E70027F1E7200001F01AFB00281FD0C1
:10265000002E1DDD7319882647190193B60020004E
:1026600001F086FD5A3080002018406801358188CD
:102670000430090A023101F0A3FC200001F048FDFA
:10268000A3590133A351BD4202D0019B9D42E6D123
:10269000114BE35C002BABD095239B00E35C002B3C
:1026A000A6D00E4BE15A0029A2D00D4AA35C994254
:1026B00002D90133A3549BE700231A212000A3541D
:1026C00001F02EFB94E7C046300DFF1F3409FF1FB9
:1026D00000140340E010FF1F5A02000072020000C5
:1026E0005E020000F8B51D4B1D4F1A78002A10D16C
:1026F000BA7B002A02D101321A7003E0032AFAD011
:10270000022AF8D001F0BCFB00220120154B1A7000
:10271000F8BD154B154D1C68154B9E7801232B7089
:102720002878C0B200F0DEFCBB7B002B0BD101F09F
:1027300087FCA1239B007343E41883239B00E418C8
:1027400023782B70E4E7032B02D101F079FBF0E74B
:102750000020022BDCD101F083FCEAE71C09FF1FFB
:10276000A60BFF1F2309FF1F3409FF1F490AFF1F84
:10277000300DFF1FF0B587B00EAD2F780FAD2D785F
:102780000593AC46634614000E4D0CAA12782E78C1
:1027900003930D9B009201932200059B029701F089
:1027A0003FFB2E70012C01D0042C08D18022064959
:1027B0008B889343054A1278D20113438B8007B06C
:1027C000F0BDC0461C09FF1F6C11FF1F7809FF1FD9
:1027D0000B001B3B70B504003020E02B0DD813001C
:1027E000E025493BFF3B9BB2ED00AB4205D8034BD4
:1027F000200019825A8201F0EBFA70BD8410FF1F8D
:1028000010B501F0D5FC054B00205B68052B04D901
:10281000034A5268D20200D4980810BD001000404C
:10282000FCE100E070B501F033FB0D4B1B68FC339D
:10283000DC691D6AFFF7E4FF6419844204D2094B86
:1028400001241B68002B07D004220024064B1A70B9
:10285000064A93690133936101F06AFB200070BD61
:10286000A465FF1F9809FF1F2309FF1FFC0FFF1F0F
:1028700070B50C4D2B68FC335C6A01F009FBFFF767
:10288000BFFF2B680025FC339B6AE318834204D208
:10289000054B1B68AB4200D1051B01F049FB28002A
:1028A00070BDC046A465FF1F9809FF1FD722044BC7
:1028B00092009B5810B5002B00D0984710BDC04621
:1028C0000000FF1FF0B587B001F046F9FFF7EEFFFB
:1028D000CA4BCB4C04931B78022B45D1C94B1B68C8
:1028E000186A01F07DFBC84BC84A1A60C84BC94A38
:1028F0001A60A022C84B52001A60049B187801F09D
:102900002FFCC649C64801F0DBFBC649C64801F0AA
:10291000D7FB1022C54BFF201A60802252031A6099
:10292000802292031A60802212041A6001F018FBC0
:10293000012001F0C5F9FA20400001F0B9FA582051
:1029400001F0E6F9BA4801F033FA012001F0B8FAD3
:10295000072001F0D5FB2268B64B1A4084235B00A8
:102960001343236007B0F0BD01F01AFAB24E029093
:10297000322001F035FB33681B0629D43C2001F0DE
:102980002FFB0F2001F02CFB9C4B1B78012B00D15F
:102990001EE180223368A94D134200D0A7E02B68C6
:1029A000032013432B6001F01BFB01F0F9F9029B9C
:1029B0000299C31A5A1E814200D81A00A04B1A600D
:1029C000904B19681E2353439E4A9B18CB618AE79C
:1029D00001F0E6F980239C4ADB02116803900B4367
:1029E00013602268934B994F1A40282313432360A6
:1029F000032001F0F5FA03203D6801F0F1FA3B688D
:102A00000320DB03DB0B009301F0EAFA3B68ED03E4
:102A1000DB03ED0BDB0B8E4A0193AB18C22B30D8D6
:102A2000009B9B18C22B2CD8019B9B18C22B28D82B
:102A3000009B2A009D4200D21A00009B9D4200D9B3
:102A40001D00019B934200D21300019A954200D9C8
:102A500015005B1B122B14D80C22336814209343EF
:102A6000336033687B4A1340336001F0B9FA0821C0
:102A70003B682268DB038A432260774ADB0B1360E2
:102A80007FE7032001F0ACFA3B68DB03DB0B059327
:102A900001F086F9039B0399C21A531E814200D8A4
:102AA00013006E4A93421BD9FF23356869492D0AEA
:102AB0001D4032686B1C1B060A401B0C134333601D
:102AC0000C23326800209A43083B1343336001F023
:102AD0000FFA6348634BA840984206DCFEF732FFCA
:102AE000019B009D0093059B95E75F48F6E7002357
:102AF0005E4F554A3B6080231168DB020B43136035
:102B000080222B68032013432B6001F069FA3B6895
:102B1000052601333B6080232A685B0213432B6048
:102B20002268444B03201A40514B1343236001F0A9
:102B300057FA0821454B1A682368D2038B43236058
:102B4000454B023900931B68D20B4B439A420CD879
:102B50009B1A3B2B0BD8236846490B4023602B68FC
:102B60000B402B60444B1A601FE7D31AF1E7013E7C
:102B7000F6B2002ED4D123683E4A134023602B685E
:102B800013402B603B68042B07D9BFF34F8F3B4B9F
:102B90003B4ADA60BFF34F8FFEE780222B680320A9
:102BA00093432B6001F01CFA2268224B03201A4049
:102BB00028231343236001F013FA244B009A1B6867
:102BC000DB03DB0B1360082223689343236097E742
:102BD00007222C4D2B681340012B02D1002001F05D
:102BE000BFFAAB68284A02201340AB6001F0F8F945
:102BF0008023AA685B001343AB60D6E64A0AFF1F36
:102C00005CF00040A465FF1F000003400180063D0A
:102C1000BC00034034080000A4000340710200001F
:102C200014100040FFFF3F002810004000E100E0CA
:102C30003075000000FEFEFFC4F0004044F000408C
:102C40008C65FF1F7206000040F0004064F00040F9
:102C500091FCFFFFFF00FFFF9465FF1FE30C0000E6
:102C6000E88000005F361E0060361E001444FF1F1F
:102C700028000100FFFFFEFF9065FF1F00ED00E050
:102C80000400FA053CF00040FFFEFFFF694E336888
:102C900088331B6883F3088801F0DAF900F0C4FB7D
:102CA000654B664A1B68934207D0002001F020F96B
:102CB0000221634A13688B431360FFF703FE614BE5
:102CC000614C1878C0B201F0D3F90023A36002333D
:102CD000A3605E4B0120236001F082F90323A3600F
:102CE00001F05EF8040001F063FA050001F058F805
:102CF000574B186000F0FCFF564B1968621A531EC0
:102D0000A14200D213008022D203934201D39B023E
:102D10009B0A3268D16AC90700D478E04E491C0C7E
:102D200009689BB24C4359432402090A64180327DB
:102D30004A49FC3293680A6849489B1A494A4A4EF4
:102D400012684A499B18414A34609A183B400193E3
:102D5000036892089C46019B0A6063440360042B4D
:102D600003D901323B400A6003600B684049E41814
:102D7000200001F01DF93F4F3D493B68C3183B60FF
:102D80002000019301F054F93B4C206808183849A1
:102D90002060884205D9019B01333B6001F048F96E
:102DA000216001F065F8354B1B78002B0ED001F047
:102DB000FFF93168324B4A1B1B6812189A4233D212
:102DC000591A4919091A2F4801F07AF92E4C237A19
:102DD000002B0FD001F0ECF93168E3684A1B1218A0
:102DE000934224D9591A4919091A284801F068F957
:102DF00000232372264B83F3088801F0A1F80220F8
:102E000001F0E6F8002001F073F800F041FFDC016A
:102E100099000234641A5900641A09214B43803323
:102E2000CB40A408E41882E7FA218900CBE71949CE
:102E3000DBE7C046A465FF1F0C0AFF1FB641210354
:102E400010000040490AFF1F14100040C409000090
:102E5000100AFF1F340AFF1F380AFF1F200AFF1F36
:102E6000280AFF1F1C0AFF1F8865FF1F240AFF1F77
:102E7000710200006008FF1F2C0AFF1F1C09FF1FC2
:102E8000E408FF1F00100040740BFF1F3C100040BF
:102E900000000020DC050000A022054B92009B589A
:102EA00010B5002B01D0984710BD01F069F9FBE780
:102EB0000000FF1FA122054B92009B5810B5002B6C
:102EC00001D0984710BD01F05BF9FBE70000FF1F40
:102ED000A222054B92009B5810B5002B01D09847B9
:102EE00010BD01F04DF9FBE70000FF1FA322054BC9
:102EF00092009B5810B5002B01D0984710BD01F0EF
:102F00003FF9FBE70000FF1FA422054B92009B58EE
:102F100010B5002B01D0984710BD01F031F9FBE747
:102F20000000FF1F70B501F043F9514B18600420F9
:102F300001F04EF800F07CFF0400C30702D400F05B
:102F4000DFFE70BD00224B4B1A604B4B18780138E6
:102F500004282CD800F076FE03231B1F2700200036
:102F600001F0B6F80128ECD0444C2378042B71D141
:102F700001F096F8002806D001F0DAF8582000F0A9
:102F8000C7FE02232370032001F022F8D9E72000B6
:102F900000F0EEFEE6E7200001F02AF8E2E720006C
:102FA00000F0DEFEDEE7200000F092FFDAE700F03E
:102FB000CFFE0500012808D1314B1B78053B012BC2
:102FC00003D82000FFF768FFCEE72C4B1B78022BBD
:102FD00001D0052B20D1022D28D12A4B9B7BAB435E
:102FE0001CD12000FFF766FF254B18780128BBD1C4
:102FF0006405B9D4234925224B7B034205D1233AEA
:1030000013405A42534126331A000B7D9342ABD9E9
:10301000322000F085FFA7E7022D07D1184B1B785F
:10302000052B11D12000FFF753FFDDE7012D0BD158
:10303000012B03D12000FFF759FF95E7062B03D1A1
:103040002000FFF761FF8FE7200001F099F8022DC3
:103050008AD1C9E7032B04D10B4B987C01F060F8AF
:1030600091E7072B8FD1094B987B00F039FF8AE756
:103070009C09FF1F9809FF1F9009FF1F2309FF1FCD
:103080001C09FF1FA60BFF1FBC0BFF1FD40BFF1F4C
:10309000FA210A4B0A4A49001A640A4A5A500A4A53
:1030A00004395A50094A08319A64094A5A50094A5F
:1030B0005C315A50084ADA667047C0460000FF1F6C
:1030C0007527FF1F7128FF1F2528FF1F7D23FF1F66
:1030D000E526FF1F011EFF1FD51DFF1F10B500F0C5
:1030E00099FD10BD8023F7B59C46264B264F0193D2
:1030F0002649274A274D284C284B02281AD16046DA
:1031000038600868264E3040802636033043086019
:1031100001990978002909D11660224A2A60224AB9
:103120002260E02219689143A03A1BE08021C90285
:103130001160F2E766463E600F68194E3E408027F8
:10314000FF023E430E600199097800290DD11760F6
:1031500001280ED1154A2A60154A2260E02219681A
:103160009143C03A0A431A60F7BD80218902116079
:10317000EEE7E0210F4A02432A600F4A22601A68F4
:103180008A43F0E74B0AFF1FE0000340D8000340EA
:103190009000034000000340500003404000034003
:1031A000FFFFE3FF0280063D804508220180063DC7
:1031B000806608220080069880550822F8B51E4BCC
:1031C00080261A68002014003440324232D11A6836
:1031D0001A4F32431A6001223B68063093433B602A
:1031E00000F0FEFE0122164D2B681E432E603B6848
:1031F0000A2613433B608027BF00124B1B683B42EB
:1032000011D1013EF6B2FF2E09D17E220E4B1C6871
:103210002B68E40B1440934323432B6005E0082004
:1032200000F0DEFEE9E7002EEFD180222B68600877
:1032300093432B60F8BDC046C4F000405CF00040F2
:1032400018F0004068F0004060F0004010B500F059
:1032500047FF01215820034A00F012FFFFF7AEFF9D
:1032600010BDC046600AFF1F10B578220021034838
:1032700000F03EFF00F094FF002010BDAC68FF1F7F
:1032800070B5040000F004FE00230C200B4A01007E
:1032900059438D18515C00290DD0A14208D101235A
:1032A00000246B7000F0ACFE00F042FE200070BD08
:1032B00001330A2BEBD11224F6E7C046AC68FF1F9E
:1032C00070B5040000F0E4FD002319001D000D4A54
:1032D0001078002806D0A0420CD1557001310C3274
:1032E0000A29F5D1002B0AD100F05AFF00F020FE88
:1032F000002070BD5078461EB0411B18EEE700F06C
:103300007FFEF3E7AC68FF1FF7B504000C20002335
:1033100084460E4D019267465F43E85D7E19A042E8
:1033200012D000280BD10A4B9C4662461B7808330A
:103330001370019B70707C557160B360FEBD0133EA
:103340000A2BE8D10320F9E70720F7E7AC68FF1F55
:10335000A868FF1F8021204BC9051B6870B58B60D2
:103360001E4BC1241A680123FF2013434B611C4BE1
:10337000A4001A681B4B00251A601B4B1A681B4BD4
:103380001A601B4B1A5982431A51C52292009C584D
:103390008443BF38204398509C58164804408020EE
:1033A000C001204398509858134C0002000A014372
:1033B0009950124B1B78DB08AB4201DC002070BD3A
:1033C0002378002B06D0A368002B00D09847013546
:1033D0000C34EEE71220F2E7AC44FF1FA844FF1FB5
:1033E000B0F00040A468FF1FB4F00040A068FF1FC9
:1033F00000E100E0FF00FFFFAC68FF1FA868FF1FAF
:10340000030010B51F2809D8072200201340072405
:1034100004490A78A24313430B7010BD0023062011
:10342000F5E7C046A868FF1F034A04491368002057
:103430000B4013607047C0461CF00040FFFFC1FF07
:10344000054B06491B780A6805485B0702401B0BC1
:10345000134300200B607047A868FF1F1CF000405A
:10346000FFFFC1FF70B50C25FFF7EAFF0A4B1C7880
:103470000A4BE4086543ED18002C01D1200070BD13
:103480002B78002B06D06B68002B00D09847013CAE
:103490000C3DF1E71220F2E7A868FF1FA068FF1FAC
:1034A00007B50422074801A900F034F9019B013354
:1034B00005D18023044ADB0411680B43136000200C
:1034C0000EBDC0461C18001114F00040F0B50500F8
:1034D0002026184B87B00493049B002B03D11124A2
:1034E000200007B0F0BD002102220B0001910091E5
:1034F000052000F055FD02230F490A681A42FCD14D
:103500000596059C631E0593002CFAD10B4A13689F
:10351000002BFCDA0F276F440121380000F078FC03
:103520003B782B42DCD0052000F05AFD049B013B88
:103530000493D1E7FFFFFF0790C8004000C8004098
:1035400007B500F0A5FC80220821D205936A0191FD
:10355000002B01D10739916202210C4A11600199B7
:10356000481E01900029FAD1033111600531019103
:103570000199481E01900029FAD11160002B02D157
:103580008022D205936200F0D3FC07BD00C000404A
:10359000F0B52D4C89B02378002B4FD1FEF7B2F94E
:1035A00002232A4F03903A681A42FCD12023069343
:1035B000069B5A1E0692002BFAD1254E3368002B2B
:1035C000FCDA0120FFF782FF011E02D0112009B0B2
:1035D000F0BD030003220190009005AD9F2000F094
:1035E000DFFC0321280000F013FC02233A681A4292
:1035F000FCD120230793079B5A1E0792002BFAD178
:103600003368002BFCDA0120FFF760FF0028DDD1D2
:103610000398FEF78BF9AA786B7811041B020B4311
:1036200029780B4363601300113B0A49052B07D827
:1036300001239340A3600B60012323700020C6E7A1
:1036400080231B03F6E7C0469444FF1F90C8004048
:1036500000C800409808FF1F1E4B30B55A68187804
:103660001D4B85B0D31859424B41012100930023D3
:1036700000F0A6FB194B1A4A02259A6300221A652C
:1036800010325A658022C4219D65164B1648D2021D
:10369000DA6789004258154B80241A4080231B04A6
:1036A00013434350642341200393E40500F078F969
:1036B000402000F075F96562039D6B1E0393002D99
:1036C000FAD103236362FFF73BFFA562FFF760FFB8
:1036D00005B030BDA044FF1F95FFFEF700C80040B5
:1036E000050001FF04E100E000E100E0FFFF00FF52
:1036F00010B5064B18705960FFF7AEFF002113207C
:10370000034AFFF701FE002010BDC046A044FF1F82
:103710005936FF1FF0B5040085B003920291FEF701
:10372000F1F8882263035B0B52051A438023DB0503
:103730009D6A8023274F0092BA68002601901B03E0
:103740009A420CD9F82326001B041E401C4206D0C6
:103750008022214B52025E6219680A431A60002DD2
:103760000BD100F095FB02221C4B1A608023DB0575
:103770005A62013A9A6200F0DBFB0023039A9342FB
:1037800020D1002D0AD100F083FB144B03221D60D1
:103790008023DB055A629D6200F0CAFB8023BA6871
:1037A0001B039A4208D9002E06D000220A4B0C496E
:1037B0005A621A680A401A600198FEF7B7F80020AA
:1037C00005B0F0BD009A0299D2181278CA5401339C
:1037D000D4E7C0469444FF1F00C8004000C000402A
:1037E000FFFFFEFFF0B587B0029103920400FEF7E1
:1037F00089F8019000F04CFB802302250122234E22
:10380000DB0535605D629A6200F092FB204F3B68F9
:103810002B42FCD120230493049B5A1E0492002BBC
:10382000FAD11C4D2B68002BFCDA0120FFF74EFE6D
:10383000002802D0112007B0F0BD2000039A0299A1
:1038400000F066FB022304003A681A42FCD12023F0
:103850000593059B5A1E0592002BFAD12B68002B6D
:10386000FCDA0120FFF732FE051EE3D100F010FB69
:1038700080230322DB0535605A629D6200F058FB0D
:103880000198FEF753F8E0B2D5E7C04600C000400B
:1038900090C8004000C80040F0B5802687B0040002
:1038A000FEF730F8F605B36A02250393029000F0A4
:1038B000EFFA0123244F3D607562B36200F038FBDC
:1038C000224E33682B42FCD120230493049B5A1EC2
:1038D0000492002BFAD11E4D2B68002BFCDA01203C
:1038E000FFF7F4FD002802D0112007B0F0BD200042
:1038F00000F0D6F90223019032681A42FCD120234D
:103900000593059B5A1E0592002BFAD12B68002BBC
:10391000FCDA0320FFF7DAFD041EE5D100F0B8FA67
:1039200080230322DB053C605A629C6200F000FBAE
:10393000039B002B01D1FFF703FE0298FDF7F6FF72
:103940006B461879D1E7C04600C0004090C80040DF
:1039500000C8004007B5000201910422000A01A935
:10396000FFF740FF0EBD000073B5050005240B4AAC
:10397000A3005B429B1819686B46DE1D300000F007
:10398000DFFB022804D133782B55013CEFD276BD02
:10399000052CFCD00128FAD10230F8E714090011F7
:1039A0001F2807D8012380228340D20591680B434A
:1039B000936070473F2808D8012380222038834035
:1039C000D20551690B435361F3E75F28F1D8012316
:1039D000802240388340D205116A0B431362E8E726
:1039E0001F2807D8012280218240C9058B68934394
:1039F0008B6070473F2808D8012280212038824000
:103A0000C9054B6993434B61F3E75F28F1D8012265
:103A1000802140388240C9050B6A93430B62E8E776
:103A20001F2810D880230200DB05153A1968012AE7
:103A300006D820229143196019680A431A6070471A
:103A400001228240F6E73F2811D880230200DB05DF
:103A5000353AD968032A06D810229143D960D9682B
:103A60000A43DA60EBE7012220388240F5E75F285D
:103A7000E5D842238022181A413B8340D205516A7F
:103A800099435162516A0B435362D8E710B5040061
:103A9000012813D1A022184992050B685B015B092C
:103AA00013430B60154B164A19681140154A0A4317
:103AB0001A60402219680A431A6010BD0028FCD120
:103AC00001000A2000F0C4F921000B2000F0C0F929
:103AD000C0220A4B920019680A4340211A601A68F2
:103AE0008A431A60B022044912060B685B015B0925
:103AF00013430B60E1E7C04614F000401CF00040A7
:103B00007F00FEFF80FD010072B6074A1368013393
:103B100013600422054B1A600023054A13608022BB
:103B2000D2055360FEE7C0467808FF1FC0F0004092
:103B3000C4F00040044B054A1A60054B1A6000228D
:103B4000044B1A607047C046140AFF1F841E000011
:103B5000380AFF1FC4F000400023034A1360034AE1
:103B60001360034A1360704754F0004040F1004076
:103B700044F10040002310B5184C8AB00093019323
:103B80002378012B27D06946012000F0F9F900289D
:103B900017D1009B12490293019B06AA0393114B74
:103BA00002A81B680493104B1B68059300F0D0FA21
:103BB00010220E4906A800F0C3F8002804D1FF2304
:103BC000237000200AB010BD0123094A074902A84A
:103BD000237000F0BDFA0120F4E7C046A865FF1F7E
:103BE00010290011082900110C29001120290011A9
:103BF000AC65FF1F13B501246946012000F0C0F930
:103C0000034B00940193FFF7B5FF200016BDC0469B
:103C1000BB0B000010B5FFF79FFFFFF7EBFF00287D
:103C200002D0024B984710BDFEE7C046E1A200005B
:103C300002B4714649084900095649008E4402BC45
:103C40007047C04602B4714649084900095C490002
:103C50008E4402BC7047C04603B471464908400018
:103C60004900095A49008E4403BC70470000000017
:103C700001B40248844601BC604700BFE927000048
:103C800001B40248844601BC604700BF71B0000027
:103C900001B40248844601BC604700BF8552010060
:103CA00001B40248844601BC604700BFA96F01000F
:103CB00001B40248844601BC604700BF21440000B3
:103CC00001B40248844601BC604700BF691101008D
:103CD00001B40248844601BC604700BF85C10000B2
:103CE00001B40248844601BC604700BF09B000111E
:103CF00001B40248844601BC604700BFC1660100B0
:103D000001B40248844601BC604700BFDD0A0100DF
:103D100001B40248844601BC604700BF791201002B
:103D200001B40248844601BC604700BF53B900009B
:103D300001B40248844601BC604700BFE90B0100A2
:103D400001B40248844601BC604700BFCD4C01006D
:103D500001B40248844601BC604700BFDD0C01008D
:103D600001B40248844601BC604700BFF53501003C
:103D700001B40248844601BC604700BF0934010019
:103D800001B40248844601BC604700BF8937010086
:103D900001B40248844601BC604700BFCD0C01005D
:103DA00001B40248844601BC604700BF156B0100A6
:103DB00001B40248844601BC604700BF8D11010078
:103DC00001B40248844601BC604700BFC56D0100D4
:103DD00001B40248844601BC604700BF116E000078
:103DE00001B40248844601BC604700BFE9D400002A
:103DF00001B40248844601BC604700BFBD5C0100BD
:103E000001B40248844601BC604700BF0D52010066
:103E100001B40248844601BC604700BF3D71010007
:103E200001B40248844601BC604700BF9D6A00009F
:103E300001B40248844601BC604700BFBD0B0100CD
:103E400001B40248844601BC604700BF75F8000019
:103E500001B40248844601BC604700BFF99B0011D1
:103E600001B40248844601BC604700BF6D0B0100ED
:103E700001B40248844601BC604700BFD54401003C
:103E800001B40248844601BC604700BFA9D80000C5
:103E900001B40248844601BC604700BF75A9000018
:103EA00001B40248844601BC604700BFA1AF0000D6
:103EB00001B40248844601BC604700BF851201007E
:103EC00001B40248844601BC604700BFE51201000E
:103ED00001B40248844601BC604700BFF9350100C7
:103EE00001B40248844601BC604700BFC1F700002E
:103EF00001B40248844601BC604700BF016C010068
:103F000001B40248844601BC604700BFF9ED0000DF
:103F100001B40248844601BC604700BF95730100AC
:103F200001B40248844601BC604700BF613701000C
:103F300001B40248844601BC604700BF9DA900004F
:103F400001B40248844601BC604700BF7997000075
:103F500001B40248844601BC604700BFC1A500000F
:103F600001B40248844601BC604700BFED6B01000C
:103F700001B40248844601BC604700BFB35201004F
:103F800001B40248844601BC604700BFE1AC0000B8
:103F900001B40248844601BC604700BFE94C0100FF
:103FA00001B40248844601BC604700BF496D01006E
:103FB00001B40248844601BC604700BF090E0000FE
:103FC00001B40248844601BC604700BFC11501002E
:103FD00001B40248844601BC604700BF19070100D4
:103FE00001B40248844601BC604700BF018900005B
:103FF00001B40248844601BC604700BF053401009B
:1040000001B40248844601BC604700BF21A90000FA
:1040100001B40248844601BC604700BF8D820000A5
:1040200001B40248844601BC604700BFF9A6000005
:1040300001B40248844601BC604700BF090E00007D
:1040400001B40248844601BC604700BFE9F60000A5
:1040500001B40248844601BC604700BFC9A9000002
:1040600001B40248844601BC604700BF19FA000051
:1040700001B40248844601BC604700BF89140100B6
:1040800001B40248844601BC604700BF01670100DB
:1040900001B40248844601BC604700BF8B52010056
:1040A00001B40248844601BC604700BF01D700004C
:1040B00001B40248844601BC604700BF8944000047
:1040C00001B40248844601BC604700BF2D6C01006A
:1040D00001B40248844601BC604700BF01340100BE
:1040E00001B40248844601BC604700BFED6801008E
:1040F00001B40248844601BC604700BFB70E00000F
:1041000001B40248844601BC604700BFF90D0100BC
:1041100001B40248844601BC604700BF59760100E3
:1041200001B40248844601BC604700BF4DF900005D
:1041300001B40248844601BC604700BF6DF6000030
:1041400001B40248844601BC604700BF89380011B1
:1041500001B40248844601BC604700BFDD3F000057
:1041600001B40248844601BC604700BFEDA50000D1
:1041700001B40248844601BC604700BFD9B00000CA
:1041800001B40248844601BC604700BFE917010042
:1041900001B40248844601BC604700BF51B800002A
:1041A00001B40248844601BC604700BFADAE0000C8
:1041B00001B40248844601BC604700BFC95C0100ED
:1041C0000200000022B9001101000000F0B6001149
:1041D000020000001EB90011010000000042FF1F94
:1041E00002000000F8B60011010000000463FF1F88
:1041F000020000001CB90011030000007862FF1FDC
:10420000120000000200000022B9001101000000AD
:1042100038B70011020000001EB9001101000000B3
:1042200035B700110200000042B700110300000082
:10423000B362FF1F020000001CB900110300000060
:10424000C862FF1F020000001EB90011010000003B
:1042500034B700110200000040B700110300000055
:104260008962FF1F020000001CB90011030000005A
:10427000AA62FF1F0200000022B900110100000025
:104280007CB70011020000001EB9001101000000FF
:104290004943FF1F020000008EB70011010000001B
:1042A00073B70011020000001EB9001101000000E8
:1042B0004843FF1F020000008CB7001101000000FE
:1042C000D062FF1F020000001EB9001101000000B3
:1042D0004743FF1F020000008AB7001101000000E1
:1042E00063B70011020000001EB9001101000000B8
:1042F0004643FF1F0200000088B7001101000000C4
:104300005EB70011020000001EB90011010000009C
:104310004543FF1F0200000086B7001101000000A6
:1043200059B70011020000001EB900110100000081
:104330004443FF1F0200000084B700110100000089
:1043400054B7001102020202020200008D4900115E
:1043500089490011D0B70011900118001800FFFF23
:104360000701020304050602010600000000000028
:10437000000000000000000000000000000000003D
:1043800000000000000003000200000022B900113C
:104390000100000050B80011020000001EB9001119
:1043A00001000000F843FF1F020000005AB800118E
:1043B00001000000FE62FF1F020000001CB9001196
:1043C000030000005865FF1F020000001EB9001125
:1043D00001000000F843FF1F0200000058B8001160
:1043E000010000000063FF1F020000001CB9001163
:1043F000030000005065FF1F1200000000010000D4
:1044000000000111FFFF0000504859360000000075
:104410000000000001000000E1B700110B000500E2
:10442000F7000000B4000028002800283075A00024
:10443000A000A000A00000080008E001F0001000AB
:10444000100010001000100010005000500050002C
:1044500010001000D0070000000000000F00010055
:104460000500307507001000010081FF000000000A
:10447000FF000000F16D0011F96B00118969001156
:10448000FFFF0100FF000000ED970011699500118A
:1044900081940011000000000000000000000800EE
:1044A000040000003B0001085902E00188212800B7
:1044B000FF0000000200000022B90011010000000E
:1044C000E8B90011020000001EB90011010000004F
:1044D0003145FF1F020000001AB900110100000061
:1044E0006469FF1F020000001EB9001101000000F6
:1044F0003045FF1F0200000018B900110100000044
:104500002E45FF1F020000001EB90011010000002F
:104510002C45FF1F0200000016B900110100000029
:104520002445FF1F1800180000009001020000033E
:10453000020200000200000022B900110100000088
:10454000FCB90011020000001EB9001101000000BA
:104550007445FF1F0200000014B9001100000000A4
:1045600000000000020000001CB900110300000060
:064570008469FF1F20FF1B
:040000051FFF184180
:00000001FF
